:10000000A2C20000D1C20000CFC20000CDC20000D9
:10001000CBC20000C9C20000C7C20000C5C20000B8
:10002000C3C20000C1C20000BFC20000BDC20000C8
:10003000BBC20000B9C20000B7C20000B5C20000D8
:10004000B3C200000C940512AFC20000ADC20000A4
:100050000C94D825A9C20000A7C200000C942A1055
:10006000A3C200000C944D0E0C94240E9DC20000FF
:100070009BC2000099C2000097C2000095C2000018
:100080000C94D81191C200008FC200008DC20000F4
:100090008BC2000089C2000087C2000085C2000038
:1000A00083C2000081C200000C94AB117DC200002D
:1000B0007BC2000079C2000077C200000C947E1160
:1000C00073C2000071C200006FC200006DC2000068
:1000D0006BC2000069C2000067C2000065C2000078
:1000E00063C200007E0C810C700C740C7A0CB80C8E
:1000F000850C890C8F0C930C970C9D0CA10CA50CF6
:10010000B80CAB0CAF0CB30C162C232C2C2C352CB0
:10011000422C4B2CE72FE72FE72FE72FE72F582C08
:10012000652C722CE72F7F2C882C912C9E2CA72CD1
:10013000B02CB92CC22CCB2CE72FD42CDD2CE62CE8
:10014000E72FE72FE72FEF2CF82C012DE72FE72FD4
:100150000A2D172DE72FE72FE72F242D312D3E2DC8
:10016000E72F4B2D542D5D2DE72FE72FE72F662D21
:100170006F2D782DE72F852D922D9F2DE72FE72FBF
:10018000E72FAC2DB92DC62DE72FD32DE02DED2D6A
:10019000E72FE72FE72FFA2D072E142EE72F212E1A
:1001A0002A2E332EE72FE72FE72FE72FE72FE72F12
:1001B000E72FE72FE72FE72FE72FE72FE72FE72F8F
:1001C000E72FE72FE72FE72FE72FE72FE72FE72F7F
:1001D000E72F572E602E692EE72F722E7B2E842E4E
:1001E000E72FE72FE72F8D2E9A2EA72EE72FB42E7D
:1001F000C12ECE2EE72FE72FE72FDB2EE82EF52E90
:10020000E72F022F0B2F142FE72FE72FE72F1D2F9C
:10021000262F2F2FE72FE72FE72FE72FE72FE72FA7
:10022000E72FE72FE72FE72FE72F3C2E452E4E2E07
:10023000E72FE72FE72FE72FE72FE72FE72FE72F0E
:10024000E72FE72FE72FE72FE72FE72FE72FE72FFE
:10025000E72FE72FE72FE72FE72FE72FE72FE72FEE
:10026000E72FE72FE72FE72FE72FE72FE72FE72FDE
:10027000E72FE72FE72FE72FE72FE72FE72FE72FCE
:10028000E72FE72FE72FE72FE72FE72FE72FE72FBE
:10029000E72FE72FE72FE72FE72F382F412F4E2F9C
:1002A000E72F5B2F642F712FE72FE72FE72F7E2F8C
:1002B000872F942FE72FA12FAA2FB72FE72FE72FF4
:1002C000E72FC42FCD2FDA2FB033B533BA33C43371
:1002D000CE334734D833E033E833F233FC330634DB
:1002E00015341F344734293433343D344E414E499C
:1002F0004E495459494E46CDCCCC3D0AD7233C17E4
:10030000B7D13877CC2B329595E6241FB14F0A0030
:100310000020410000C84200401C4620BCBE4CCA20
:100320001B0E5AAEC59D7400407A10F35A00A0729D
:100330004E18090010A5D4E80000E8764817000020
:10034000E40B54020000CA9A3B000000E1F50500EE
:100350000080969800000040420F000000A0860137
:10036000000000102700000000E803000000006407
:1003700000000000000A0000000000010000000072
:10038000002C76D888DC674F0823DFC1DFAE59E147
:10039000B1B796E5E3E453C63AE651997696E8E6B6
:1003A000C28426EB898C9B62ED407C6FFCEFBC9C89
:1003B0009F40F2BAA56FA5F490055A2AF75C936B9B
:1003C0006CF9676DC11BFCE0E40D47FEF520E6B556
:1003D00000D0ED902E0300943577050080841E0830
:1003E0000000204E0A000000C80C333333330F984E
:1003F0006E12831141EF8D2114893BE65516CFFE15
:10040000E6DB18D1844B381BF77C1D901DA4BBE4A0
:1004100024203284725E228100C9F124ECA1E53DE2
:100420002700000A0B02090C0D0E08070304010047
:1004300000000000000000000000000000000000BC
:100440000000000000000000000000000012111079
:10045000000000000000000000000000000000009C
:100460000000000000000000002100240027002AF6
:10047000002D003000330001010000040107010AD3
:100480000100002200250028002B002E003100343E
:100490000002010000050108010B010000200023FB
:1004A00000260029002C002F00320000010000036C
:1004B00001060109010505050507050808080802E8
:1004C0000202020A0A0808040404040101010101ED
:1004D0000101010303030303030303040707070CDC
:1004E0000C0C0C0C0C0C0C02020202060606060692
:1004F0000606060B0B0B0B0B0B0B0B01021020203F
:100500000808102040102040800201020108040267
:1005100001010204081020408080402010080402DD
:100520000180040201804020100804020108040236
:10053000010102040810204080010204081020403C
:100540008000C847C34711241FBECFEFD1E2DEBFF2
:10055000CDBF00E00CBF17E0A0E0B2E0E2EAF3EAB2
:1005600000E00BBF02C007900D92A234B107D9F78B
:100570002CE0A2E4B7E001C01D92A23FB207E1F770
:1005800012E0C2EAD2E000E006C021970109802F04
:10059000FE010E94B350C13AD10780E00807A9F7D5
:1005A0000E942C3D0C94C0512BCD2F923F924F9224
:1005B0005F926F927F928F929F92AF92BF92CF92F3
:1005C000DF92EF92FF920F931F93CF93DF93CDB7FC
:1005D000DEB7E6970FB6F894DEBF0FBECDBF1C01A5
:1005E0002A013B010B871C872D873E872E960EAD77
:1005F0001FAD2E97FC01EF59FD4F60817181828103
:1006000093810E94094E9B01AC01C301B2010E947B
:10061000684E0E945F506B8B7C8B8D8B9E8BF101A3
:10062000EB59FD4F60817181828193810E94094E57
:100630009B01AC016B857C858D859E850E94684EF3
:100640000E945F506B8F7C8F8D8F9E8FF101E759D9
:10065000FD4F60817181828193810E94094E9B01CF
:10066000AC01C701B6010E94684E0E945F506F8FB7
:1006700078A389A39AA30E941E106B877C878D871D
:100680009E87F101EE51FE4F118210823296118247
:1006900010823E96A114B10461F0C501A0E0B0E063
:1006A000408151816281738184179507A607B7073E
:1006B00014F0A080B180F101EA50FE4F8114910442
:1006C00061F0C401A0E0B0E040815181628173819A
:1006D00084179507A607B70714F080809180F10171
:1006E000E650FE4F0115110561F0C801A0E0B0E031
:1006F000408151816281738184179507A607B707EE
:1007000014F000811181310120E1620E711CC501DC
:10071000A0E0B0E0F10180A791A7A2A7B3A72101B3
:10072000FAE84F0E511CA12CB12CD20158968D9293
:100730009D92AD92BC925B974101BCEF8B1ABEEFCC
:100740009B0A20E030E0F401008F118F228F338F5D
:100750000E94DA180E94DA180E94DA180E94DA1849
:1007600040914A0750914B0760914C0770914D079B
:100770004BAB5CAB6DAB7EAB0E94DA1880914E0741
:1007800090914F07A0915007B09151078F87988B98
:10079000A98BBA8B0E94DA18A0905207B090530729
:1007A000C0905407D0905507F101E359FD4F1082D6
:1007B0001182128213823496108211821282138265
:1007C0003496108211821282138234961182108222
:1007D00032961182108232961182108232964BA983
:1007E0005CA96DA97EA9408351836283738334968B
:1007F0008F859889A989BA8980839183A283B383DD
:100800003496A082B182C282D3822F96EFAC2F970A
:100810000B891C892D893E89C3010E949D2688234E
:10082000F9F085E393E00E94E53B8FEE95E00E94AE
:10083000E53BF101EE5AFF4F608171818281938126
:10084000E15FFD4F20813181428153810E94354F0C
:10085000CA01B9010E94313C0E94DA180E94E417D3
:100860006096EFAC60970B8D1C8D2D8D3E8D4F8566
:10087000588969897A89C2010E949D268823F9F0E6
:1008800081E393E00E94E53B8FEF95E00E94E53B1A
:10089000F101E453FF4F6081718182819381E756BA
:1008A000FE4F20813181428153810E94354FCA0120
:1008B000B9010E94313C0E94DA180E94E417619647
:1008C000EFAC61970F8D18A129A13AA1B601A5013E
:1008D000C4010E949D268823F9F08DE293E00E94D6
:1008E000E53B8FE096E00E94E53BF101EA5BFE4FBD
:1008F0006081718182819381ED5DFE4F2081318124
:10090000428153810E94354FCA01B9010E94313C96
:100910000E94DA180E94E417D10151961C92F1014D
:10092000E557FF4F1082E658FF4F1082C1010E9429
:100930008713C1010E948913C3010E94EB2AC201DF
:100940000E94EB2AC4010E94EB2AF101E751FE4FFD
:10095000FCA3EBA381E090E0918380837101F5E13A
:10096000EF1AFEEFFF0AD7018D939C93810103518B
:100970001E4FF8019183808341E050E0B301C10133
:100980000E943219D7014D915C91B201C1010E94C0
:100990003219F80140815181B401C1010E9432191C
:1009A00011E0F101E253FD4F1083C3010E9488263C
:1009B000C2010E948826C4010E94882664E670E075
:1009C00080E090E00E94E60FC1018A519E4FDC0159
:1009D0001C9311961C93A10148515E4FFA0110839C
:1009E0002F96FFAD2F97F1110FC060962FAD609736
:1009F000211105C061963FAD6197332339F1910113
:100A000021593F4FF90110826096FFAD6097F111B7
:100A100005C0910127513F4FF90110826196FFAD4A
:100A20006197F11105C091012D593E4FF9011082D6
:100A30002F962FAD2F97FC01208360963FAD6097D6
:100A40003C936196EFAD6197DA01EC93C3010E948C
:100A50004628C2010E944628C4010E944628C301BC
:100A60000E949C27C2010E949C27C4010E949C27CF
:100A70000E94DA18DC011C968C918F87A12CB12C76
:100A8000F101EA51FE4FFC8BEB8B910129513E4F56
:100A90003C8F2B8FA10148515E4F58A34F8FC1014E
:100AA00087519E4F9CA78BA7D101A551BE4FBEA7D2
:100AB000ADA73796F8ABEFA7255731403AA729A73E
:100AC0004F535F4F5AAB49AB815291409EA38DA3C8
:100AD000A95AB109B8A7AFA3EB89FC89808181111C
:100AE0000BC0AB8DBC8D8C91811106C0EF8DF8A130
:100AF0008081882309F44EC3FF85F1114BC34BA5B8
:100B00005CA5B301C1010E9489194DA55EA5B20182
:100B1000C1010E9489194FA558A9B401C1010E94C1
:100B20008919C3010E940628C2010E940628C40137
:100B30000E940628E9A5FAA58081882321F1C30136
:100B40000E944628A9A9BAA98C918823C9F06101FD
:100B5000B3E6CB1ABDEFDB0A7101E2E4EE1AEDEF6A
:100B6000FE0A810105571D4F910121583D4FA101FA
:100B700043595D4FB10162587E4FC3010E94CB12B1
:100B8000A9A5BAA51C92F101E451FF4F80818823E9
:100B900031F1C2010E944628F101E655FD4F8081E6
:100BA0008823C9F06101BFE5CB1ABDEFDB0A7101F3
:100BB000E0E4EE1AEDEFFE0A810101571D4F9101AD
:100BC0002D573D4FA1014F585D4FB10164567E4FE7
:100BD000C2010E94CB12F101E451FF4F1082F101DA
:100BE000EA59FE4F8081882331F1C4010E944628D2
:100BF000F101E555FD4F80818823C9F06101FBE5D6
:100C0000CF1AFDEFDF0A71012EE3E21A2DEFF20A8F
:100C100081010D561D4F910129573D4FA1014B58A0
:100C20005D4FB10166547E4FC4010E94CB12F101A9
:100C3000EA59FE4F1082810101591F4FD8018C9152
:100C4000882309F43CC0F101E956FD4F60817181B0
:100C5000072E000C880B990B0E94094E9B01AC01DA
:100C6000F101E359FD4F60817181828193810E947E
:100C70009050181624F5D8011C9264E274E08101AA
:100C800008521E4FC8018ED76BED74E0C8018AD799
:100C90006CE973E0C80186D72F96BFAD2F97BB23B1
:100CA00009F47AC3F101E258FE4F108A118A128AC0
:100CB000138AE053F1401082118212821382810163
:100CC00007511F4FF8018081882309F43CC0E0558B
:100CD000FE4F60817181072E000C880B990B0E94DA
:100CE000094E9B01AC01F101EF58FD4F608171810C
:100CF000828193810E94905018162CF5F801108281
:100D000064E274E0810108521E4FC8014BD763E0D2
:100D100075E0C80147D76CE973E0C80143D7609616
:100D2000FFAD6097FF2309F43BC3F101E456FE4F8A
:100D3000108A118A128A138AADA1BEA11D921D923A
:100D40001D921C92139781010D591E4FF80180814D
:100D5000882309F43CC0E85CFE4F60817181072E56
:100D6000000C880B990B0E94094E9B01AC01F1010C
:100D7000EB58FD4F60817181828193810E94905078
:100D800018162CF5D8011C9264E274E08101085217
:100D90001E4FC80107D76BE275E0C80103D76CE9A5
:100DA00073E0C801FFD66196BFAD6197BB2309F41C
:100DB000FBC2F101E654FE4F108A118A128A138A8F
:100DC000AFA1B8A51D921D921D921C92139760E0D1
:100DD000C3010E941527882369F0F101E25BFF4FF0
:100DE0001082118212821382E05DFE4F108A118AF6
:100DF000128A138A60E0C2010E941527882369F0D5
:100E0000EDA1FEA11082118212821382F101E4563B
:100E1000FE4F108A118A128A138A60E0C4010E9470
:100E20001527882371F0AFA1B8A51D921D921D92C0
:100E30001C921397F101E654FE4F108A118A128A10
:100E4000138AF101E159FF4F8081EB89FC8980838E
:100E5000F101E751FF4F8081AB8DBC8D8C93E6583B
:100E6000FF4F8081EF8DF8A18083F101E25BFF4F9E
:100E700020813181428153812F83388749875A8766
:100E8000ADA1BEA14D915D916D917C91EFA1F8A5B1
:100E9000C080D180E280F3804BAB5CAB6DAB7EABAE
:100EA0000E94DA188F819885A985BA8580934A07B0
:100EB00090934B07A0934C07B0934D070E94DA180C
:100EC0004BA95CA96DA97EA940934E0750934F078B
:100ED00060935007709351070E94DA18C09252072E
:100EE000D0925307E0925407F0925507C1010E9437
:100EF0008713AB89BC898C91882309F44AC00E946E
:100F00001E102B853C854D855E856217730784070F
:100F1000950760F40E941E102B853C854D855E85EB
:100F20006217730784079507A0F51EC00E941E1064
:100F30006B017C012B853C854D855E85C21AD30AE9
:100F4000E40AF50AF101EB5AFD4F2081318142811B
:100F50005381A8EEB3E00E94514F6C157D058E05BC
:100F60009F0508F425C2D6CF0E941E106B017C019C
:100F7000F101EB5AFD4F2081318142815381A8EE6E
:100F8000B3E00E94514F6C157D058E059F0508F456
:100F90000FC2AB8DBC8D8C91882309F44AC00E948E
:100FA0001E102B853C854D855E856217730784076F
:100FB000950760F40E941E102B853C854D855E854B
:100FC0006217730784079507A0F51EC00E941E10C4
:100FD0006B017C012B853C854D855E85C21AD30A49
:100FE000E40AF50AF101E75AFD4F2081318142817F
:100FF0005381A8EEB3E00E94514F6C157D058E051C
:101000009F0508F4E8C1D6CF0E941E106B017C0139
:10101000F101E75AFD4F2081318142815381A8EED1
:10102000B3E00E94514F6C157D058E059F0508F4B5
:10103000D2C1AF8DB8A18C91882309F446C0FED7E8
:101040002B853C854D855E85621773078407950760
:1010500058F4F4D72B853C854D855E856217730760
:101060008407950790F51DC0E9D76B017C012B859E
:101070003C854D855E85C21AD30AE40AF50AF10162
:10108000E35AFD4F2081318142815381A8EEB3E0C4
:101090000E94514F6C157D058E059F0508F4AEC169
:1010A000D8CFCCD76B017C01F101E35AFD4F2081F1
:1010B000318142815381A8EEB3E00E94514F6C15FB
:1010C0007D058E059F0508F499C188EA9BE026D32B
:1010D0001816190674F588EA9BE0FED28F7D8534D8
:1010E000910539F56DE974E0C10188529E4F5AD5DA
:1010F00082E693E00E94E53B0E94DA180E94E41722
:10110000F101E159FF4F1082E658FF4F1082E65877
:10111000FF4F1082AB89BC891C92EB8DFC8D108235
:10112000AF8DB8A11C92B1E0BF87AA24A394B12CC3
:1011300003C0A114B10479F062EB74E0C1018852DC
:101140009E4F30D5EB89FC891082AB8DBC8D1C92F3
:10115000EF8DF8A11082C1010E949B3BF101EC517F
:10116000FE4F808191810196918380838D329140E1
:101170000CF4B2CCD101A452BE4F8D919C91119729
:10118000892B09F0A9CC14968D919C91892B09F497
:1011900048C1A2CC810104521E4FD8018D919C916F
:1011A000892B21F0C1010E949B3BF7CF82EC94E098
:1011B0000E94E53B2F96BFAD2F97BB2309F1A114E9
:1011C000B104F1F4EF85E11140C08DE193E00E949C
:1011D000E53B0E94DA180E94E4176096FFAD609725
:1011E000FF2371F189E193E00E94E53B0E94DA1848
:1011F0000E94E41761962FAD6197211118C025C098
:1012000060963FAD6097332339F0A114B10421F407
:101210004F8541111AC0E6CF61965FAD61975523A6
:10122000A1F0A114B10489F48F8581110EC085E16C
:1012300093E00E94E53B0E94DA180E94E41705C083
:101240006196EFAD6197E111F2CF85E090E0ABA13F
:10125000BCA18D939C93910125513E4F3C872B87D8
:10126000D9018D939C93810103511E4FF801918305
:10127000808345E050E0B301C1010E943219AB8583
:10128000BC854D915C91B201C1010E943219F801F7
:1012900040815181B401C1010E943219C1010E94F3
:1012A0008B13F101E25BFF4F4081518162817381B9
:1012B000E658FF4F80819181A281B3818F8B988FF7
:1012C000A98FBA8FE658FF4FC080D180E280F380AB
:1012D0004BAB5CAB6DAB7EAB0E94DA184BA95CA943
:1012E0006DA97EA940934A0750934B0760934C0722
:1012F00070934D070E94DA182F89388D498D5A8DC9
:1013000020934E0730934F07409350075093510757
:101310000E94DA18C0925207D0925307E092540705
:10132000F0925507C1010E948713C1010E948913E1
:101330000E94DA180E943718C1010E94C119ABA19E
:10134000BCA11D921C92EB85FC8511821082D801F4
:101350001D921C9240E050E0B301C1010E9432197D
:10136000EB85FC8540815181B201C1010E94321997
:10137000D8014D915C91B401C1010E943219C101A3
:101380000E948B13BF85BB2309F43DC10E94DA186C
:1013900021E0FC01248737C1AA24A394B12C8FCC6F
:1013A000AA24A394B12CCFCCAA24A394B12C0FCD02
:1013B00069E273E0810108521E4FC801F3D36CE962
:1013C00073E0C801EFD363E575E0C801EBD322E019
:1013D000A22EB12CDECD65E273E0810108521E4FD2
:1013E000C801E0D36CE973E0C801DCD368E675E0BE
:1013F000C801D8D392E0A92EB12C1BCE61E273E0D4
:10140000810108521E4FC801CDD36CE973E0C801B9
:10141000C9D36DE775E0C801C5D382E0A82EB12C11
:1014200054CE11821082F101EE51FE4F80819181E4
:10143000009741F46EE573E0810108521E4FC80128
:10144000B1D3BDC0019709F0CAC00E94DA188C015F
:10145000FC0180819181A281B381181619061A06B8
:101460001B0644F081E090E0A0E0B0E0808391832F
:10147000A283B383F80184819581A681B781181670
:1014800019061A061B0644F081E090E0A0E0B0E0E7
:1014900084839583A683B783F80180859185A2858F
:1014A000B385181619061A061B0644F081E090E071
:1014B000A0E0B0E080879187A287B3876EE973E0F0
:1014C000CE010196ADD36EEB74E0CE0101966AD3E6
:1014D0006FEE75E0CE01019665D360914A07709179
:1014E0004B0780914C0790914D070E94094E6B016C
:1014F0007C01D8016D917D918D919C910E94094E46
:101500009B01AC01C701B6010E94F74FAB01BC01C2
:10151000CE01019617D36FEF75E0CE01019642D34D
:1015200060914E0770914F0780915007909151073D
:101530000E94094E6B017C01F801648175818681EE
:1015400097810E94094E9B01AC01C701B6010E9420
:10155000F74FAB01BC01CE010196F4D26FE076E00B
:10156000CE0101961FD3609152077091530780916D
:101570005407909155070E94094E6B017C01D801D8
:1015800018966D917D918D919C911B970E94094EAB
:101590009B01AC01C701B6010E94F74FAB01BC0132
:1015A000CE010196CFD2BE016F5F7F4F81010852FD
:1015B0001E4FC80105D389819A810E94F1480E947B
:1015C000DA18BC01CE0101960E949E17BE016F5F22
:1015D0007F4FC801F5D289819A810E94F148F101BB
:1015E000EE51FE4F808191810196823091051CF46D
:1015F0009183808302C011821082F101E052FE4F7C
:101600001182108269CA80ED94E00E94E53BC50119
:101610000E94583C8CE993E00E94E53B0E94DA1856
:10162000B0924507A0924407C501E6960FB6F8941C
:10163000DEBF0FBECDBFDF91CF911F910F91FF9005
:10164000EF90DF90CF90BF90AF909F908F907F9062
:101650006F905F904F903F902F900895CF92DF92C0
:10166000EF92FF920F931F93CF93DF936C017A0158
:101670008B01C0E0D0E0CE15DF0589F0D8016D9177
:101680008D01D601ED91FC910190F081E02DC60114
:101690001995892B11F47E0102C02196ECCFC70168
:1016A000DF91CF911F910F91FF90EF90DF90CF903E
:1016B0000895089580E090E00895FC01538D448DD5
:1016C000252F30E0842F90E0821B930B541710F0ED
:1016D000CF96089501970895FC01918D828D9817FA
:1016E00061F0828DDF01A80FB11D5D968C91928D06
:1016F0009F5F9F73928F90E008958FEF9FEF089503
:10170000FC01918D828D981731F0828DE80FF11DCB
:10171000858D90E008958FEF9FEF0895FC01918DE6
:10172000228D892F90E0805C9F4F821B91098F73DF
:101730009927089588EA9BE0F1DF21E0892B09F4DD
:1017400020E0822F0895FC01848DDF01A80FB11DD8
:10175000A35ABF4F2C91848D90E001968F739927E7
:10176000848FA689B7892C93A089B1898C918064D4
:101770008C93938D848D981306C00288F389E02D95
:1017800080818F7D80830895EF92FF920F931F9346
:10179000CF93DF93EC0181E0888F9B8D8C8D981324
:1017A00005C0E889F989808185FD23C0F62E0B8D5F
:1017B00010E00F5F1F4F0F731127E02E8C8DE81282
:1017C0000BC00FB607FCFACFE889F989808185FF45
:1017D000F5CFCE01B8DFF2CF8B8DFE01E80FF11D02
:1017E000E35AFF4FF0820B8FEA89FB898081806288
:1017F00007C0EE89FF896083E889F9898081806468
:10180000808381E090E0DF91CF911F910F91FF9055
:10181000EF900895CF93DF93EC01888D8823C1F07A
:10182000EA89FB89808185FD05C0A889B9898C91E9
:1018300086FD0EC00FB607FCF5CF808185FFF2CF85
:10184000A889B9898C9185FFEDCFCE017CDFE8CFE7
:10185000DF91CF91089580E090E0892B19F06ADF45
:10186000811125C080E090E0892B41F080E090E07C
:10187000892B21F00E94000081111CC080E090E0C3
:10188000892B41F080E090E0892B21F00E9400003C
:10189000811113C080E090E0892BA1F080E090E0FE
:1018A000892B81F00E94000081110AC008950E94D6
:1018B0000000D8CF0E940000E1CF0E940000EACFD4
:1018C0000C940000089590E0FC013197E231F1059D
:1018D00008F04EC08827EE58FF4F8F4F0C94B3503E
:1018E000809180008F7703C0809180008F7D8093EE
:1018F0008000089580918000877FF9CF84B58F772D
:1019000002C084B58F7D84BD08958091B0008F772B
:1019100003C08091B0008F7D8093B00008958091C6
:1019200090008F7707C0809190008F7D03C08091D9
:101930009000877F8093900008958091A0008F771A
:1019400007C08091A0008F7D03C08091A000877F99
:101950008093A0000895809120018F7707C0809127
:1019600020018F7D03C080912001877F809320011B
:1019700008953FB7F89480918F0B9091900BA091B0
:10198000910BB091920B26B5A89B05C02F3F19F083
:101990000196A11DB11D3FBFBA2FA92F982F8827EF
:1019A000820F911DA11DB11DBC01CD0142E0660F4A
:1019B000771F881F991F4A95D1F708950E94A35158
:1019C0000C94F1480C94F1480F931F93CF93DF933D
:1019D000EC0188819981009729F02A813B812617A3
:1019E000370788F48B016F5F7F4F0E94BB500097D1
:1019F00061F0998388831B830A832C813D81232B8B
:101A000011F4FC01108281E001C080E0DF91CF91F0
:101A10001F910F9108958F929F92AF92BF92CF9294
:101A2000DF92EF92FF920F931F930E942E1762E0B6
:101A300070E00E94C736892BD1F40E942E1721E056
:101A40002F931F921F921F921F92812C912CA12CD9
:101A5000B12CC12CD12C760197018601B701A601CA
:101A60000E94D5020F900F900F900F900F9080E082
:101A700090E01F910F91FF90EF90DF90CF90BF907B
:101A8000AF909F908F9008958F929F92AF92BF9248
:101A9000CF92DF92EF92FF920F931F930E942E1727
:101AA0001F9221E02F931F921F921F92812C912C45
:101AB000A12CB12CC12CD12C760197018601B70144
:101AC000A6010E94D5020F900F900F900F900F90DB
:101AD00080E090E01F910F91FF90EF90DF90CF900A
:101AE000BF90AF909F908F900895EF92FF920F93C9
:101AF0001F93CF93DF93FC0124813581611571051C
:101B000011F480E018C041155105A1F07B01EC01F2
:101B10008A01020F131FB80157DF882391F3288130
:101B200039818C819D81B701820F931F0E94B95129
:101B30001D830C8381E0DF91CF911F910F91FF9066
:101B4000EF900895EF92FF920F931F93CF93DF933F
:101B5000CDB7DEB764970FB6F894DEBF0FBECDBF2A
:101B60007C01CB01BA018E010F5F1F4F22E044E0E0
:101B70000E943D48BC01FC0101900020E9F731972B
:101B8000AF01481B590BC701B0DF64960FB6F8943C
:101B9000DEBF0FBECDBFDF91CF911F910F91FF90A0
:101BA000EF9008956115710549F0FB010190002047
:101BB000E9F73197AF01461B570B97CF80E00895A7
:101BC000FB0144815581608171818FCFEF92FF923B
:101BD0000F931F93CF93DF93EC017B018A01BA012E
:101BE000F3DE2881398181110DC02115310519F0ED
:101BF000C9010E94F148198218821D821C821B8231
:101C00001A8206C01D830C83B701C9010E94B95115
:101C1000CE01DF91CF911F910F91FF90EF9008952A
:101C2000FC011182108213821282158214826115C6
:101C3000710549F0FB0101900020E9F73197AF01F0
:101C4000461B570BC3CF08951F920F920FB60F92EA
:101C500011240BB60F922F933F934F935F936F9383
:101C60007F938F939F93AF93BF93EF93FF9388EAF4
:101C70009BE069DDFF91EF91BF91AF919F918F91B3
:101C80007F916F915F914F913F912F910F900BBE7C
:101C90000F900FBE0F901F9018951F920F920FB6C6
:101CA0000F9211240BB60F922F938F939F93EF9364
:101CB000FF93E091B80BF091B90B8081E091BE0BDE
:101CC000F091BF0B82FD12C090818091C10B8F5F9C
:101CD0008F732091C20B821751F0E091C10BF0E09D
:101CE000E855F44F958F8093C10B01C08081FF911F
:101CF000EF919F918F912F910F900BBE0F900FBE80
:101D00000F901F901895CF93DF93282F30E0F901A3
:101D1000EF5DFB4F8491F901E550FB4FD491F90140
:101D2000EB54FB4FC491CC2389F08111CCDDEC2F17
:101D3000F0E0EE0FFF1FE556FB4FA591B491EC913B
:101D4000ED2381E090E021F480E002C080E090E0AB
:101D5000DF91CF9108951F93CF93DF93282F30E029
:101D6000F901EF5DFB4F8491F901E550FB4FD491F0
:101D7000F901EB54FB4FC491CC23C1F0162F811114
:101D8000A2DDEC2FF0E0EE0FFF1FEF57FB4FA59108
:101D9000B4918FB7F894111105C09C91ED2FE09587
:101DA000E92302C0EC91ED2BEC938FBFDF91CF9133
:101DB0001F910895CF92DF92EF92FF920F931F939E
:101DC000CF93DF936C018B017A01EC01CA57D44F9A
:101DD000888187FF04C0FB011182108224C08CE03F
:101DE0008C9D90018D9D300D11248881A901480F93
:101DF000511D87FD5A958091DD0C90E048175907D9
:101E000094F48881A901480F511D87FD5A95CA0194
:101E1000FA01EE0FFF1F8E0F9F1FFC01E35BF34FD4
:101E2000808186FD19C088818F5F88838CE08C9DBE
:101E300090018D9D300D11248881A901480F511DFD
:101E400087FD5A958091DD0C90E048175907B4F44E
:101E500088818C303CF112C08881280F311D87FDAC
:101E60003A95F901EE0FFF1F2E0F3F1FF901E35BBB
:101E7000F34F808160E08F736EDFD5CFF8018081F2
:101E80009181049680349C4918F480E49CE904C054
:101E9000F801808191810496F701918380838FEF0F
:101EA000888344C0F801408151818881B901680F5D
:101EB000711D87FD7A95CB01FB01EE0FFF1F8E0F81
:101EC0009F1FFC01E35BF34F81819281840F951F7B
:101ED000F701918380838881A901480F511D87FDF7
:101EE0005A95CA01FA01EE0FFF1F8E0F9F1FFC01CA
:101EF000E35BF34F808186FF19C08881280F311D75
:101F000087FD3A95F901EE0FFF1F2E0F3F1FF901D4
:101F1000E35BF34F808161E08F73DF91CF911F917D
:101F20000F91FF90EF90DF90CF9015CFDF91CF9181
:101F30001F910F91FF90EF90DF90CF900895CF9376
:101F4000DF9390E0FC01E550FB4F2491FC01EB5442
:101F5000FB4F8491882361F190E0880F991FFC0169
:101F6000E959FB4FC591D491FC01EF57FB4FA59167
:101F7000B491611109C09FB7F8948881209582239C
:101F80008883EC912E230BC0623061F49FB7F894E4
:101F90003881822F809583238883EC912E2B2C937C
:101FA0009FBF06C08FB7F894E8812E2B28838FBF80
:101FB000DF91CF9108958230910538F0880F991FF5
:101FC000880F991F05970197F1F708958F929F92B7
:101FD000AF92BF92CF92DF92EF92FF926B017C01A2
:101FE000C8DC4B015C01C114D104E104F104E9F047
:101FF000C0DCDC01CB0188199909AA09BB09883E1C
:102000009340A105B10578F321E0C21AD108E10897
:10201000F10888EE880E83E0981EA11CB11CC11443
:10202000D104E104F10421F7DECFFF90EF90DF90BF
:10203000CF90BF90AF909F908F9008952FB7F89456
:1020400060918B0B70918C0B80918D0B90918E0B0E
:102050002FBF08951F920F920FB60F9211242F9346
:102060003F938F939F93AF93BF9380918B0B9091EE
:102070008C0BA0918D0BB0918E0B30918A0B23E0CD
:10208000230F2D3720F40196A11DB11D05C026E8B0
:10209000230F0296A11DB11D20938A0B80938B0BF9
:1020A00090938C0BA0938D0BB0938E0B80918F0B24
:1020B0009091900BA091910BB091920B0196A11D64
:1020C000B11D80938F0B9093900BA093910BB093C5
:1020D000920BBF91AF919F918F913F912F910F9054
:1020E0000FBE0F901F901895CF92DF92EF92FF9244
:1020F000CF93DF93EC01603282E078070CF03DC0B3
:1021000077FD06C0653B71052CF064EB70E002C002
:1021100060E070E0898128E830E06901C81AD108E0
:1021200087FDD394CC0CDD1CCC0CDD1C0D2C000CDD
:10213000EE08FF088A8128E532E0281B310987FD77
:102140003395220F331F220F331FC901330FAA0B00
:10215000BB0B9C01AD012C193D094E095F09DB0148
:102160000E945B4F24EB30E040E050E00E94354F8E
:10217000C20ED31EE41EF51EB6018881803380F5A1
:10218000998148E850E0491B510997FD5395440F48
:10219000551F440F551F6417750784F09A8128E571
:1021A00032E0291B310997FD3395220F331F220F8F
:1021B000331FAB01261737070CF4A9014250510910
:1021C000440F551F2FB7F89490E0FC01EE0FFF1F4E
:1021D0008E0F9F1FFC01E35BF34F528341832FBFA0
:1021E000DF91CF91FF90EF90DF90CF9008951F93F4
:1021F000CF93DF93EC01162F8881803308F04DC018
:1022000061E0812F9CDE8881E82FF0E09F01220FA2
:10221000331FE20FF31FE35BF34F1F739081907C3A
:10222000192B108319821A826CE00E94A7509CE03F
:10223000899FB001112440E050E09A01260F371F1A
:10224000F901EE0FFF1F2E0F3F1FF901E35BF34F64
:10225000908196FD16C04F5F5F4F4C30510569F776
:10226000813001F51092800082E08093810010920D
:10227000850010928400B19A80916F0082608093F3
:102280006F00E881F0E0CF01880F991FE80FF91F78
:10229000E35BF34F8081806480838881DF91CF91FD
:1022A0001F910895823061F4109290008093910004
:1022B000109295001092940088BB80937100E1CF3A
:1022C000833069F41092A00082E08093A100109204
:1022D000A5001092A40089BB80937200D2CF811117
:1022E000D0CF1092200182E080932101109225012D
:1022F000109224018ABB80937300C3CF1F920F9268
:102300000FB60F9211240BB60F922F933F934F935A
:102310005F936F937F938F939F93AF93BF93EF934D
:10232000FF9348E251E064E271E080E090E042DD3A
:10233000FF91EF91BF91AF919F918F917F916F919D
:102340005F914F913F912F910F900BBE0F900FBE59
:102350000F901F9018951F920F920FB60F92112495
:102360000BB60F922F933F934F935F936F937F938F
:102370008F939F93AF93BF93EF93FF9348EA50E0FF
:1023800064EA70E083E090E015DDFF91EF91BF918A
:10239000AF919F918F917F916F915F914F913F91FD
:1023A0002F910F900BBE0F900FBE0F901F9018959E
:1023B0001F920F920FB60F9211240BB60F922F930C
:1023C0003F934F935F936F937F938F939F93AF93BD
:1023D000BF93EF93FF9348E950E064E970E082E037
:1023E00090E0E8DCFF91EF91BF91AF919F918F91C9
:1023F0007F916F915F914F913F912F910F900BBE05
:102400000F900FBE0F901F9018951F920F920FB64E
:102410000F9211240BB60F922F933F934F935F931C
:102420006F937F938F939F93AF93BF93EF93FF939C
:1024300048E850E064E870E081E090E0BBDCFF91A8
:10244000EF91BF91AF919F918F917F916F915F912C
:102450004F913F912F910F900BBE0F900FBE0F9099
:102460001F90189508950F931F93CF93DF93FC014E
:102470002081318121153105D1F1EC01822F43DC1E
:1024800021E0892B09F420E02B876A85261729F0A3
:102490001E821F82188619860BC08E819F81A88597
:1024A000B9850196A11DB11D8E839F83A887B98729
:1024B0000E811F81288539858A819B81AC81BD81F0
:1024C000081719072A073B0794F081E068278881DD
:1024D00042DC0990D881C02D0E946F3540E050E069
:1024E000BE01DF91CF911F910F910C94D932DF91F2
:1024F000CF911F910F910895CF92DF92EF92FF92AB
:102500000F931F93CF93DF937C016B018A01E90145
:102510000E944732F601EE0FFF1FEE0FFF1FEA5A2F
:10252000F84F80819181F701918380830E94473227
:10253000000F111F000F111FF801EA5AF84F81E038
:10254000408151816281738141305105610571057E
:1025500009F080E0F70182870E944732CC0FDD1F2F
:10256000CC0FDD1FCA5AD84F88819981AA81BB81BF
:10257000F70182839383A483B58316821782108622
:102580001186DF91CF911F910F91FF90EF90DF9017
:10259000CF90089508952F923F924F925F926F923D
:1025A0007F928F929F92AF92BF92CF92DF92EF92E3
:1025B000FF920F931F93CF93DF9300D000D0CDB73E
:1025C000DEB79E838D834B015A013A83298318011C
:1025D000FC82EB82FA01408051806280738020E0AF
:1025E00030E0A901C301B2010E949050181674F4A2
:1025F000F6012081318142815381C301B2010E94E1
:10260000924FF5016083718382839383ED81FE8114
:10261000E05AFF4F8081F401028D138DC088D1886C
:10262000E288F388F1014080518062807380D80194
:10263000A7019601882341F00E945B4F6415750540
:102640008605970544F023C00E945B4F4616570647
:1026500068067906E4F4F501408051806280738059
:1026600020E030E04AEF56E4C301B2010E94034E7D
:1026700087FF0DC020E030E040E85FE3C301B20116
:102680000E94934FF5016083718382839383D80105
:10269000A70196010E945B4FF101608371838283E1
:1026A00093830D811E81025C1F4FF801808191810F
:1026B000A281B381E981FA8180839183A283B3836C
:1026C000EB81FC8180819181892B41F0C4010E94C2
:1026D0007936F801608371838283938326960FB6DF
:1026E000F894DEBF0FBECDBFDF91CF911F910F9148
:1026F000FF90EF90DF90CF90BF90AF909F908F9022
:102700007F906F905F904F903F902F90089552D59B
:1027100098C750D56BC4CF93DF93EC01FC01E25313
:10272000FD4F1082EE58F1098081811104C0CE0165
:1027300040960E947426FE01EF5BFD4F808181115F
:1027400005C0CE0186579F4F0E947426FE01EE5BA6
:10275000FD4F8081811105C0CE018C5F9E4F0E948C
:10276000742664E670E080E090E0DF91CF912ECC9B
:10277000662319F08DEA93E002C086EA93E00C9498
:10278000E53B0C94F1480C94F148AF92BF92CF9284
:10279000DF92EF92FF920F931F93CF93DF93EC01A1
:1027A00086E390E09E8B8D8B87E390E0988F8F8BF4
:1027B00086E290E09A8F898F8AE190E09C8F8B8FE0
:1027C0008CE190E09E8F8D8F88E190E098A38F8FB1
:1027D00083E090E09AA389A382E090E09CA38BA37E
:1027E000FE01E657FF4F8CE390E0968385838DE3EF
:1027F00090E09087878388E390E0928781871486B2
:10280000138616861586108A17868EE090E0928BC6
:10281000818B8FE090E0948B838BE658FF4F8EE2A4
:1028200090E09683858380E390E0908787838EE3B2
:1028300090E0928781871486138616861586108A03
:10284000178682E190E0928B818B83E190E0948BFC
:10285000838BEB51FF4F11821082329611821082CE
:10286000329611821082CE010E948A1DCE0165D758
:102870006E0182E8C81A8EEFD80AAA24A394B12C5C
:10288000F601B58EA48E7E01F4E6EF1AFEEFFF0A84
:1028900084E090E0F701958F848F8E0106541E4FDF
:1028A00088E090E0F801958F848F80E190E0F60158
:1028B0009183808381E190E0958384838FE190E030
:1028C0009383828381E290E097838683C6010E948E
:1028D0001336F601828580878385818787E190E0C2
:1028E000F7019183808389E190E09583848383E27B
:1028F00090E09383828385E290E097838683C7018B
:102900000E941336F70182858087838581878BE15A
:1029100090E0F801918380838DE190E0958384833A
:1029200087E290E09383828389E290E097838683B5
:10293000C8010E941336F8018285808783858187CC
:10294000E65FFE4F80819181729740815181628163
:102950007381369720813181F601318F208F448B2E
:10296000558B668B778B019729F48FEF9FEF938FB1
:10297000828F03C0F601B38EA28EFE01EA53FD4F93
:1029800080819181709740815181628173813897F4
:1029900020813181F701318F208F448B558B668BDD
:1029A000778B019719F48FEF9FEF03C081E090E0E0
:1029B000F701938F828FFE01E853FD4F8081918153
:1029C0003E974081518162817381C055DD4F2881DE
:1029D0003981F801318F208F448B558B668B778B33
:1029E000019719F48FEF9FEF03C081E090E0F801A9
:1029F000938F828FDF91CF911F910F91FF90EF9076
:102A0000DF90CF90BF90AF9008952F923F924F925A
:102A10005F926F927F928F929F92AF92BF92CF926E
:102A2000DF92EF92FF920F931F93CF93DF93CDB777
:102A3000DEB7CA57D1090FB6F894DEBF0FBECDBFBF
:102A40008C01FC0110821182128213821482158281
:102A500016821782108611861286138614861586B2
:102A6000168617862C01F0E14F0E511CC2010E9400
:102A70000D2B68018AE8C80ED11CC6010E940D2BDF
:102A80007801ECEFEE1AEEEFFE0AC7010E940D2B63
:102A90003801F2E86F1AFEEF7F0AC3010E94A336E5
:102AA000480184E6881A8EEF980AC4010E94A33672
:102AB0005801E6E4AE1AEEEFBE0AC5010E94A33645
:102AC0006EE973E0C80188529E4FAAD8F801E2521D
:102AD000FE4F11821082329611821082329611823C
:102AE00010823296118210823296108231961082B4
:102AF00031961082319611821082329611821082A4
:102B0000329611821082329610823196108231965E
:102B100010823196108211821282138234961082B2
:102B200011821282138234961082118212821382D1
:102B3000349610821182128213823496108211828E
:102B4000128213823496108211821282138234967A
:102B500010821182128213823496108211821282A4
:102B6000138234961082118212821382349610825C
:102B70001182128213823496108211821282138281
:102B8000349610821182128213823496108211823E
:102B9000128213823496108211821282138234962A
:102BA0001082118212821382349610823196108222
:102BB00031961082319610821182128213823496DD
:102BC0001082118212821382349610821182128234
:102BD000138234961082319610823196108231968B
:102BE0001082319610823196108231961082319681
:102BF0001082319610823196108231961082319671
:102C00001082319610823196108231961082319660
:102C10001082319610823196108231961082319650
:102C20001082319610823196108231961082319640
:102C30001082319610821182128213823496108291
:102C400011821282138234961082118212821382B0
:102C5000D801AF59BD4F8CE0E9E3F3E001900D924C
:102C60008A95E1F7F801E359FD4F10821182128233
:102C7000138234961082118212821382349610824B
:102C8000118212821382349611821082329611823E
:102C90001082329611821082329610821182128234
:102CA000138234961082118212821382349610821B
:102CB0001182128213823496108211821282138240
:102CC00034961082118212821382349610821182FD
:102CD00012821382349611821082329611821082EF
:102CE00032961182108232961082118212821382E1
:102CF00034961082118212821382349610821182CD
:102D0000128213823496108231961082319610828C
:102D1000319611821082329611821082329611827F
:102D2000108232961082118212821382349610829F
:102D300011821282138234961082118212821382BF
:102D4000349611821082329611821082329611824C
:102D5000108232961182108232961182108232963F
:102D60001182108232961182108232961182108264
:102D70001801F2E32F1AFDEF3F0AF1011082CE0194
:102D800001960E940D2B8AE7FE013196D201019037
:102D90000D928A95E1F7CE0101960E940D2B8AE7EC
:102DA000FE013196D60101900D928A95E1F7CE0190
:102DB00001960E940D2B8AE7FE013196D701019002
:102DC0000D928A95E1F788E5F801808B89E5F60197
:102DD00080838AE5F7018083CE0101960E94A336A5
:102DE0008EE1FE013196D30101900D928A95E1F7B3
:102DF000CE0101960E94A3368EE1FE013196D401E8
:102E000001900D928A95E1F7CE0101960E94A336BA
:102E10008EE1FE013196D50101900D928A95E1F780
:102E2000C801B3DCF1011082C658DF4F0FB6F89429
:102E3000DEBF0FBECDBFDF91CF911F910F91FF90ED
:102E4000EF90DF90CF90BF90AF909F908F907F904A
:102E50006F905F904F903F902F900895CF93DF93A6
:102E600080919D0B90919E0B892B51F48FEC92E0F9
:102E70000E945C48EC01C9DDD0939E0BC0939D0B72
:102E800080919D0B90919E0BDF91CF9108954F9271
:102E90005F926F927F928F929F92AF92BF92CF92EA
:102EA000DF92EF92FF920F931F93CF93DF9300D0A7
:102EB0001F92CDB7DEB7FB011689078982889388F8
:102EC000A684B784C284D384E484F5844680578082
:102ED00060847184428153816481758149835A83FE
:102EE0006B837C83BBDF1F921F921F920F931F93F4
:102EF0009301820149815A816B817C810E94D502B4
:102F00000F900F900F900F900F9080E090E00F9037
:102F10000F900F900F90DF91CF911F910F91FF9025
:102F2000EF90DF90CF90BF90AF909F908F907F9069
:102F30006F905F904F90089508950895EF92FF92DB
:102F40000F931F93CF93DF93CDB7DEB72E970FB6B6
:102F5000F894DEBF0FBECDBF8C016EE973E00E9416
:102F6000100E62E975E0C8010E94D20D609146071B
:102F70007091470780914807909149072AE0AE0178
:102F80004F5F5F4F7A010E94C049F7010190002016
:102F9000E9F73197AF014E195F09B701C8010E94E7
:102FA000750D6CE973E0C8010E94D20DC8012E9620
:102FB0000FB6F894DEBF0FBECDBFDF91CF911F914A
:102FC0000F91FF90EF90089582E995E00E94E53B14
:102FD0006091460770914707809148079091490793
:102FE0000E94313C8CE993E00C94E53B0F931F93D6
:102FF000CF93DF93EC0185E995E00E94E53B89E9F9
:1030000095E00E94E53B07E91BE0F8016081CE01F5
:10301000AFDB8DE995E00E94E53BF8016181CE01CF
:10302000A7DB81EA95E00E94E53BF8016281CE01D1
:103030009FDB85EA95E00E94E53BF8016381CE01C4
:1030400097DB89EA95E00E94E53BF8016481CE01B7
:103050008FDB8DEA95E00E94E53BF8016581CE01AA
:1030600087DBCE01DF91CF911F910F91ADCFCF9232
:10307000DF92EF92FF92CF93DF93EC0188819981E9
:10308000AA81BB81181619061A061B0644F081E0B6
:1030900090E0A0E0B0E088839983AA83BB838C8111
:1030A0009D81AE81BF81181619061A061B0644F0D1
:1030B00081E090E0A0E0B0E08C839D83AE83BF838D
:1030C00088859985AA85BB85181619061A061B06D8
:1030D00044F081E090E0A0E0B0E088879987AA877B
:1030E000BB878EEB94E00E94E53B8FEE95E00E945B
:1030F000E53B60914A0770914B0780914C07909196
:103100004D070E94094E6B017C01688179818A819B
:103110009B810E94094E9B01AC01C701B6010E9430
:10312000F74F42E00E945D3C8FEF95E00E94E53B47
:1031300060914E0770914F07809150079091510711
:103140000E94094E6B017C016C817D818E819F8183
:103150000E94094E9B01AC01C701B6010E94F74FC6
:1031600042E00E945D3C8FE096E00E94E53B60916A
:1031700052077091530780915407909155070E9410
:10318000094E6B017C01688579858A859B850E9443
:10319000094E9B01AC01C701B6010E94F74F42E006
:1031A0000E945D3CCE01DF91CF91FF90EF90DF90C8
:1031B000CF900ACF8091950B9091960B892B91F52A
:1031C0008DE090E00E945C48FC01148610924A0752
:1031D00010924B0710924C0710924D0710924E0719
:1031E00010924F07109250071092510710925207F9
:1031F0001092530710925407109255071092940B97
:103200001092930B109246071092470710924807AE
:103210001092490710924507109244079093960B1D
:103220008093950B8091950B9091960B08950F9339
:103230001F93CF93DF938B01EA0181E593E00E9416
:10324000E53B8EE496E00E94E53BF80180810E9418
:10325000263CCE010E94583CADDFDF91CF911F91FB
:103260000F91B2CECF92DF92EF92FF920F931F9306
:10327000CF93DF93CDB7DEB728970FB6F894DEBFB4
:103280000FBECDBF8B016A0188529E4F7C016DE459
:1032900073E00E94D20D6EE476E0C7010E94D20D69
:1032A000F801808189831A8241E050E08E010F5F2E
:1032B0001F4FB801C7010E94750D4AE0B801C60151
:1032C0000E94B649F80101900020E9F73197AF015B
:1032D000401B510BB801C7010E94750D6BDFBC018B
:1032E000C8012CDEB801C7010E94E00D89819A81D6
:1032F0000E94F14828960FB6F894DEBF0FBECDBFEE
:10330000DF91CF911F910F91FF90EF90DF90CF90C1
:103310000895FC01DB01AD59BF4F8C91882319F052
:1033200022E030E002C020E030E0DB01AB59BF4FCB
:103330008C91882311F023E030E0DB01AC59BF4FC2
:103340008C91882311F024E030E0DB01AA59BF4FB3
:103350008C91882311F026E030E0DA018D919C9168
:103360008217930721F091E0121613060CF090E0FB
:10337000DA012D933C93992319F0A901CF0172CF63
:1033800008958F929F92AF92BF92CF92DF92EF9269
:10339000FF920F931F93CF93DF93EC0189E493E0A7
:1033A0000E94E53B8FEE95E00E94E53B6E0182E8CE
:1033B000C81A8EEFD80AC6010E9479360E94094EBB
:1033C0004B015C01FE01EF59FD4F608171818281EB
:1033D00093810E94094E9B01AC01C501B4010E947A
:1033E000F74F42E00E945D3C8FEF95E00E94E53B85
:1033F0007E01E4E6EE1AEEEFFE0AC7010E9479367E
:103400000E94094E4B015C01FE01EB59FD4F6081AA
:103410007181828193810E94094E9B01AC01C5019B
:10342000B4010E94F74F42E00E945D3C8FE096E0BD
:103430000E94E53B8E0106541E4FC8010E9479365A
:103440000E94094E4B015C01C759DD4F68817981AB
:103450008A819B810E94094E9B01AC01C501B40188
:103460000E94F74F42E00E945D3CA4DEADDD85E4A2
:1034700093E00E94E53B8FEE95E00E94E53BF6016C
:10348000A28DB38D20893189428953890E945B4F77
:103490000E94313C8FEF95E00E94E53BF701A28D41
:1034A000B38D20893189428953890E945B4F0E94E4
:1034B000313C8FE096E00E94E53BF801A28DB38D90
:1034C00020893189428953890E945B4F0E94313C97
:1034D00071DEDF91CF911F910F91FF90EF90DF9000
:1034E000CF90BF90AF909F908F906ECD4F925F9294
:1034F0006F927F928F929F92AF92BF92CF92DF9204
:10350000EF92FF920F931F93CF93DF9300D01F9200
:10351000CDB7DEB70E944732409032085090330852
:1035200060903408709035080E94473280903608C9
:1035300090903708A0903808B09039083BDEC090D2
:103540004A07D0904B07E0904C07F0904D0732DED1
:10355000C701B6010E94094E6B017C01C301B20193
:103560000E94094E9B01AC01C701B6010E94F74FB2
:103570002B013C0160914E0770914F0780915007DD
:10358000909151070E94094E6B017C01C501B40165
:103590000E94094E9B01AC01C701B6010E94F74F82
:1035A000AB01BC0149835A836B837C8357DC1F9238
:1035B0001F921F921F921F92812C912CA12CB12C33
:1035C000C12CD12C760149815A816B817C818A0181
:1035D0009B01B301A2010E94D50240DC1F921F9201
:1035E0001F921F921F9297018601B301A2010E94B0
:1035F000D50234DC1F921F921F921F921F929701D7
:103600008601B701A6010E94D5020FB6F894DEBF6D
:103610000FBECDBF80E090E00F900F900F900F9005
:10362000DF91CF911F910F91FF90EF90DF90CF909E
:10363000BF90AF909F908F907F906F905F904F90D2
:103640000895CF93DF9383E00E94830EEC01B2DDF7
:1036500091E0CD2B09F490E09093970B82E00E94CB
:10366000830EEC01A7DD91E0CD2B09F490E090935F
:10367000980B8EE00E94830EEC019CDD91E0CD2B37
:1036800009F490E09093990B8FE00E94830EEC0177
:1036900091DD91E0CD2B09F490E090939A0B82E1BB
:1036A0000E94830EEC0186DD91E0CD2B09F490E0C1
:1036B00090939B0B83E10E94830EEC017BDD91E0F4
:1036C000CD2B09F490E090939C0BDF91CF9108955E
:1036D000CF93DF93EC012AEC30E04BEC50E069EC47
:1036E00070E00E947C122EEC30E04FEC50E06DEC6C
:1036F00070E0CE010C960E947C1224ED30E045ED86
:1037000050E063ED70E0CE0148960E947C1228EDF7
:1037100030E049ED50E067ED70E0CE0184960E9404
:103720007C122EED30E04FED50E06DED70E0CE01FB
:10373000C096DF91CF910C947C122F923F924F92C2
:103740005F926F927F928F929F92AF92BF92CF9231
:10375000DF92EF92FF920F931F93CF93DF93EC01D1
:103760000E944732FE01E956FD4F80911209909167
:103770001309918380830E944732FE01E756FD4F73
:103780008091160990911709918380830E94473296
:10379000FE01E556FD4F80911A0990911B09918316
:1037A00080830E9447328E0103561D4F60913A0973
:1037B00070913B0980913C0990913D090E94094E0E
:1037C000F80160837183828393830E9447321E01D4
:1037D000FFE52F1AFDEF3F0A60913E0970913F0906
:1037E00080914009909141090E94094EF101608346
:1037F0007183828393830E94473220E030E048EC5B
:1038000052E4F80160817181828193810E94F74FB7
:103810002B013C0120E030E048EC52E4F1016081F2
:103820007181828193810E94F74F4B015C0160910D
:1038300042097091430980914409909145090E9481
:10384000094E20E030E048EC52E40E94F74F6B0153
:103850007C012AE037ED43E25CE3C301B2010E9440
:10386000905018168CF420E030E046EC52E4C3018E
:10387000B2010E94034E87FD0FC0412C512C46EC33
:10388000642E42E4742E08C05AE0452E57ED552EA2
:1038900053E2652E5CE3752EF8014082518262820C
:1038A00073822AE037ED43E25CE3C501B4010E9474
:1038B000905018168CF420E030E046EC52E4C5013C
:1038C000B4010E94034E87FD0FC0812C912C26EC81
:1038D000A22E22E4B22E08C03AE0832E37ED932EBA
:1038E00033E2A32E3CE3B32EF10180829182A282C7
:1038F000B3822AE037ED43E25CE3C701B6010E94E0
:10390000905018168CF420E030E046EC52E4C701E9
:10391000B6010E94034E87FD0FC0C12CD12C86EC4E
:10392000E82E82E4F82E08C09AE0C92E97EDD92E31
:1039300093E2E92E9CE3F92EFE01EB55FD4FC08288
:10394000D182E282F3820E9447328091FA089091FC
:10395000FB08FE01E455FD4F918380830E944732AE
:103960008091FE089091FF08FE01E255FD4F918382
:1039700080830E9447328091020990910309FE01E1
:10398000E055FD4F918380830E9447328091220948
:1039900090912309A0912409B0912509FE01EE54CC
:1039A000FD4F80839183A283B3830E94473280912D
:1039B000260990912709A0912809B0912909FE01B3
:1039C000EA54FD4F80839183A283B3830E944732E0
:1039D00080912A0990912B09A0912C09B0912D0971
:1039E000FE01E654FD4F80839183A283B3830E943E
:1039F000473280914A0990914B09FE01E254FD4FF4
:103A0000918380830E94473280914E0990914F09A3
:103A1000FE01E054FD4F918380830E9447328091E4
:103A2000520990915309FE01EE53FD4F918380831B
:103A30000E9447328091620990916309FE01EC5324
:103A4000FD4F918380830E94473280916609909157
:103A50006709FE01EA53FD4F918380830E9447323C
:103A600080916A0990916B09FE01E853FD4F9183A3
:103A700080830E9447328091EA089091EB08A091E0
:103A8000EC08B091ED08FE01E755FD4F0197A10547
:103A9000B10519F481E0808301C010820E94473291
:103AA0008091EE089091EF08A091F008B091F10894
:103AB000FE01E655FD4F0197A105B10519F481E01E
:103AC000808301C010820E9447328091F208909159
:103AD000F308A091F408B091F508C555DD4F0197A2
:103AE000A105B10519F481E0888301C01882DF9136
:103AF000CF911F910F91FF90EF90DF90CF90BF90EB
:103B0000AF909F908F907F906F905F904F903F907D
:103B10002F9008952F923F924F925F926F927F92D3
:103B20008F929F92AF92BF92CF92DF92EF92FF92CD
:103B30000F931F93CF93DF93CDB7DEB760970FB688
:103B4000F894DEBF0FBECDBF988B8F870E9447329F
:103B5000EF85F889E151FE4F81E0409122085091B4
:103B600023086091240870912508452B462B472B8C
:103B700009F480E080830E944732EF85F889E051A4
:103B8000FE4F81E040912608509127086091280857
:103B900070912908452B462B472B09F480E0808340
:103BA0000E944732EF85F889EF50FE4F81E0409147
:103BB0002A0850912B0860912C0870912D08452BF4
:103BC000462B472B09F480E080830E944732809186
:103BD000720890917308A0917408B0917508EF85F0
:103BE000F889EE50FE4F80839183A283B3830E94B5
:103BF00047328091760890917708A0917808B0912B
:103C00007908EF85F889EA50FE4F80839183A2837B
:103C1000B3830E94473280917A0890917B08A091EB
:103C20007C08B0917D08EF85F889E650FE4F8083CF
:103C30009183A283B3830E94473280914A08909176
:103C40004B08A0914C08B0914D08EF85F889E65FCC
:103C5000FD4F80839183A283B3830E94473280917A
:103C60004E0890914F08A0915008B0915108EF85EF
:103C7000F889E25FFD4F80839183A283B3830E9422
:103C800047328091520890915308A0915408B09106
:103C90005508EF85F889EE5EFD4F80839183A283FE
:103CA000B3830E94473280915A0890915B08A0919B
:103CB0005C08B0915D08EF85F889EA5EFD4F80836E
:103CC0009183A283B3830E94473280915E089091D2
:103CD0005F08A0916008B0916108EF85F889E65E01
:103CE000FD4F80839183A283B3830E9447328091EA
:103CF000620890916308A0916408B0916508EF850F
:103D0000F889E25EFD4F80839183A283B3830E9492
:103D100047328091FA079091FB07A091FC07B09180
:103D2000FD07EF85F889EE5DFD4F80839183A283C7
:103D3000B3830E9447328091FE079091FF07A091C4
:103D40000008B0910108EF85F889EA5DFD4F808396
:103D50009183A283B3830E9447328091020890919D
:103D60000308A0910408B0910508EF85F889E65D85
:103D7000FD4F80839183A283B3830E944732EF85F6
:103D8000F889E25DFD4F81E02091D2073091D307A1
:103D90002130310509F080E080830E944732EF85B1
:103DA000F889E15DFD4F81E02091D6073091D7077A
:103DB0002130310509F080E080830E944732EF8591
:103DC000F889E05DFD4F81E02091DA073091DB0753
:103DD0002130310509F080E080830E944732EF8571
:103DE000F889E45BFD4F81E04091AA075091AB0751
:103DF0006091AC077091AD07452B462B472B09F41A
:103E000080E080830E944732EF85F889E35BFD4FB5
:103E100081E04091AE075091AF076091B00770917B
:103E2000B107452B462B472B09F480E080830E9485
:103E30004732EF85F889E25BFD4F81E04091B207A0
:103E40005091B3076091B4077091B507452B462B8D
:103E5000472B09F480E080830E944732EF85F88980
:103E6000E15BFD4F81E040918208509183086091B1
:103E7000840870918508452B462B472B09F480E078
:103E800080830E944732EF85F889E05BFD4F81E037
:103E90004091860850918708609188087091890840
:103EA000452B462B472B09F480E080830E94473244
:103EB000EF85F889EF5AFD4F81E040918A085091D3
:103EC0008B0860918C0870918D08452B462B472BF1
:103ED00009F480E080830E944732EF85F889EE5A2A
:103EE000FD4F81E02091BA073091BB0721303105A9
:103EF00009F080E080830E944732EF85F889ED5A0F
:103F0000FD4F81E02091BE073091BF072130310580
:103F100009F080E080830E944732EF85F889EC5AEF
:103F2000FD4F81E02091C2073091C3072130310558
:103F300009F080E080830E9447328091820790914F
:103F40008307A0918407B0918507EF85F889EB5A24
:103F5000FD4F80839183A283B3830E944732809177
:103F6000860790918707A0918807B0918907EF8510
:103F7000F889E75AFD4F80839183A283B3830E941F
:103F8000473280918A0790918B07A0918C07B0915E
:103F90008D07EF85F889E35AFD4F80839183A283D3
:103FA000B3830E944732EF85F889E05CFD4F81E0E2
:103FB00040919207509193076091940770919507F3
:103FC000452B462B472B09F480E080830E94473223
:103FD000EF85F889EF5BFD4F81E0409196075091A6
:103FE00097076091980770919907452B462B472BAF
:103FF00009F480E080830E944732EF85F889EE5B08
:10400000FD4F81E040919A0750919B0760919C077A
:1040100070919D07452B462B472B09F480E0808348
:104020000E94473280918A0990918B09A0918C0956
:10403000B0918D09EF85F889EF5CFD4F8083918306
:10404000A283B3830E94473280918E0990918F0999
:10405000A0919009B0919109EF85F889EB5CFD4F33
:1040600080839183A283B3830E9447328091920917
:1040700090919309A0919409B0919509EF85F889E1
:10408000E75CFD4F80839183A283B3830E94473214
:10409000EF85F889ED5BFD4F81E02091EA073091D3
:1040A000EB072130310509F080E08083EF85F88946
:1040B000EC5BFD4F1082EF85F889EB5BFD4F1082C2
:1040C0000E944732EF85F889EA5BFD4F81E020913D
:1040D000E6073091E7072130310509F080E0808361
:1040E000EF85F889E95BFD4F1082EF85F889E85B81
:1040F000FD4F10820E944732EF85F889E75BFD4F44
:1041000081E020910A0830910B082130310509F037
:1041100080E080830E944732EF85F889E65BFD4F9F
:1041200081E020910E0830910F082130310509F00F
:1041300080E080830E944732EF85F889E55BFD4F80
:1041400081E020911208309113082130310509F0E7
:1041500080E080830E944732EF85F889E35CFD4F61
:1041600081E020919A0930919B092130310509F0B5
:1041700080E080830E944732EF85F889E25CFD4F42
:1041800081E020919E0930919F092130310509F08D
:1041900080E080830E944732EF85F889E15CFD4F23
:1041A00081E02091A2093091A3092130310509F065
:1041B00080E080830E9447320F8518890F591D4F78
:1041C0008091320890913308A0913408B09135085D
:1041D000F80180839183A283B3830E944732EF84E6
:1041E000F888FBE9EF1AFDEFFF0A809136089091FD
:1041F0003708A0913808B0913908F701808391837E
:10420000A283B3830E94473280913A0890913B0881
:10421000A0913C08B0913D082F85388927593D4F22
:10422000F90180839183A283B383F8014081518196
:1042300062817381141615061606170644F041E0D4
:1042400050E060E070E04083518362837383F70144
:104250004081518162817381141615061606170676
:1042600044F041E050E060E070E0408351836283BD
:104270007383181619061A061B064CF081E090E0AD
:10428000A0E0B0E0F90180839183A283B383D901D8
:104290008D909D90AD90BC90F701C080D180E28060
:1042A000F380D8014D905D906D907C900E94DA185B
:1042B000FC014082518262827382C482D582E6828E
:1042C000F78280869186A286B386EF85F889E35CC3
:1042D000FD4FB081B983EF85F889EF5CFD4F808198
:1042E0009181A281B3814F855889475B5D4FFA0167
:1042F000F081FB834F8558894E5A5D4FFA01F0815A
:10430000FA834F8558894D5B5D4FFA01F081FF8339
:104310004F8558894A5B5D4FFA01F081F8874F85D8
:104320005889415B5D4FFA01F081F9874F855889C3
:10433000445B5D4FFA01F081FA87EF85F889E25D11
:10434000FD4F2080EF85F889E151FE4F3080EF85E9
:10435000F889EB5AFD4F4081518162817381EF856D
:10436000F889EE5DFD4F0081118122813381EF8557
:10437000F889EA5EFD4FC080D180E280F380EF854E
:10438000F889E65FFD4F80809180A280B380EF8541
:10439000F889EE50FE4F4080518062807380EF8537
:1043A000F88940A651A662A673A684A695A6A6A6DD
:1043B000B7A6C0AAD1AAE2AAF3AA04AB15AB26AB52
:1043C00037AB40AF51AF62AF73AF34AE25AE2A8585
:1043D00025A3398536A34A8147A340E450E060E035
:1043E00070E0E05CFF4F40835183628373832885D4
:1043F000EF85F88926AF3F8137AFAF014C5B5F4F48
:104400002B81FA012083EF85F889EB5BFF4F8083D6
:104410009183A283B383EF85F889E75BFF4F3981EE
:104420003083AF85B88955968D919C915697863388
:10443000910589F48AEF94E2FD01E658FF4F9183DC
:10444000808332961182108288EF94E236969183AF
:104450008083329630C08C33910589F482EF94E2E8
:10446000EF85F889E658FF4F91838083EF85F889BF
:10447000E458FF4F1182108280EF94E212C08E97B1
:10448000E1F48AEE94E2EF85F889E658FF4F9183D4
:104490008083EF85F889E458FF4F1182108284EE03
:1044A00094E2EF85F889EE57FF4F91838083EF8583
:1044B000F889EC57FF4F11821082EF85F889838DC0
:1044C000948D4A97D1F486EF94E2E258FF4F91839E
:1044D0008083EF85F889E058FF4F1182108284EFC6
:1044E00094E2EF85F889EA57FF4F91838083EF8547
:1044F000F889E857FF4F11821082EF85F889E25C56
:10450000FD4F20812983EF85F889EB5CFD4F4080CA
:10451000518062807380EF85F889E65BFD4F3081C2
:104520003B83EF85F889ED5AFD4F9081EF85F8893F
:10453000EC5BFD4F40814F83EF85F889E95BFD4FD0
:1045400050815887EF85F889E05BFD4F8081EF85CA
:10455000F889E35BFD4FA081AA87EF85F889E15DCB
:10456000FD4F2080EF85F889E051FE4F3080EF85C8
:10457000F889E75AFD4F20813181428153812B8791
:104580003C874D875E87EF85F889EA5DFD4F408166
:10459000518162817381EF85F889E65EFD4FC080AD
:1045A000D180E280F380EF85F889E25FFD4F808063
:1045B0009180A280B380EF85F889E657FF4F2F8561
:1045C00038892A503E4FD9010D911D912D913C9172
:1045D000008F118F228F338F848E958EA68EB78E8B
:1045E000C0A2D1A2E2A2F3A244A355A366A377A3DB
:1045F0002B853C854D855E8520A731A742A753A713
:1046000034A625A63A85358B868B978B80E490E07F
:10461000A0E0B0E080AB91ABA2ABB3AB488546A7BE
:104620005F8157A78B8184AB45AA56AA67AA70AE53
:10463000998191AF858196818633910589F48AEFBE
:1046400094E2AF85B889AC50BF4F8D939C93AF85F2
:10465000B889AA50BF4F1D921C9288EF94E226C0E1
:104660008C33910589F482EF94E2AF85B889AC5020
:10467000BF4F8D939C93AF85B889AA50BF4F1D92B1
:104680001C9280EF94E212C08E97E1F48AEE94E2DD
:10469000AF85B889AC50BF4F8D939C93AF85B889D7
:1046A000AA50BF4F1D921C9284EE94E2AF85B88948
:1046B000A450BF4F8D939C93AF85B889A250BF4F34
:1046C0001D921C92838594854A97D9F486EF94E2D3
:1046D000EF85F889E850FF4F91838083EF85F88953
:1046E000E650FF4F1182108284EF94E2EF85F88943
:1046F000F39591838083EF85F889EE5FFE4F1182F9
:104700001082EF85F889E15CFD4FA081A9832F8598
:104710003889275C3D4FD9018D919D910D90BC91B9
:10472000A02D8B839C83AD83BE83EF85F889E55BE9
:10473000FD4FB081BA83EF85F889EC5AFD4F208197
:104740002F83EF85F889EB5BFD4F30813887EF854C
:10475000F889E85BFD4F40814987EF85F889EF5A7A
:10476000FD4F2080EF85F889E25BFD4F3080EF85BB
:10477000F889E05DFD4F3081EF85F889EF50FE4FFD
:104780002081EF85F889E35AFD4F80819181A281D4
:10479000B381EF85F889E65DFD4F408151816281EB
:1047A0007381EF85F889E25EFD4FC080D180E280A1
:1047B000F380EF85F889EE5EFD4F80809180A280C6
:1047C000B3800F8518890C5F1E4FEF85F889E6507E
:1047D000FE4F4080518062807380F801408E518E80
:1047E000628E738E848E958EA68EB78EC0A2D1A255
:1047F000E2A2F3A244A355A366A377A380A791A73F
:10480000A2A7B3A724A735A7358A268A2F81278B8D
:1048100080E490E0A0E0B0E080AB91ABA2ABB3ABA2
:10482000298526A7388537A74A8144AB8B819C818F
:10483000AD81BE8185AB96ABA7ABB0AF298121AF6F
:10484000858196818633910589F48AEF94E2EF851C
:10485000F889E259FE4F91838083EF85F889E0590A
:10486000FE4F1182108288EF94E226C08C339105AE
:1048700089F482EF94E2EF85F889E259FE4F918343
:104880008083EF85F889E059FE4F1182108280EF16
:1048900094E212C08E97E1F48AEE94E2EF85F889F3
:1048A000E259FE4F91838083EF85F889E059FE4FEE
:1048B0001182108284EE94E2EF85F889EA58FE4F67
:1048C00091838083EF85F889E858FE4F118210822A
:1048D000D8011B968D919C911C974A97E1F486EF25
:1048E00094E2EF85F889EE58FE4F91838083EF853F
:1048F000F889EC58FE4F1182108284EF94E2EF8524
:10490000F889E658FE4F91838083EF85F889E45853
:10491000FE4F11821082EF85F889E05CFD4F208107
:104920008F8598894096222311F0F2D101C0DCD105
:10493000EF85F889EF5BFD4F20818F859889865739
:104940009F4F222311F0E4D101C0CED1EF85F88929
:10495000EE5BFD4F80818823D1F0C80160960FB6D1
:10496000F894DEBF0FBECDBFDF91CF911F910F91A5
:10497000FF90EF90DF90CF90BF90AF909F908F907F
:104980007F906F905F904F903F902F90C1C1C80172
:1049900060960FB6F894DEBF0FBECDBFDF91CF910A
:1049A0001F910F91FF90EF90DF90CF90BF90AF904D
:1049B0009F908F907F906F905F904F903F902F903F
:1049C00093C18FEF9FEF0895EBE0F1E08081877F47
:1049D00080830895EBE0F1E0808188608083089512
:1049E0008E9808958E9A089514980895149A0895AB
:1049F00088980895889A08950C94F1480C94F14889
:104A00000C94F1480C94F1480C94F1480F931F93C7
:104A1000CF93DF93FB0102A113A1C68DD78D0E9416
:104A2000C632C530D105E1F064F4249771F564E035
:104A300070E08EED9CE00E94F710B8018EED9CE0D6
:104A400022C0C630D105B1F02B97F9F46BE070E0CD
:104A500087EE9CE00E94F710B80187EE9CE013C03F
:104A600065E070E081EE9CE00E94F710B80181EEF5
:104A70009CE009C066E070E084EE9CE00E94F710C4
:104A8000B80184EE9CE00E94741080E090E0DF9119
:104A9000CF911F910F9108958F929F92AF92BF92E5
:104AA000CF92DF92EF92FF920F931F930E942E17E7
:104AB0001F921F9221E02F931F921F92812C912C05
:104AC000A12CB12CC12CD12C760197018601B70104
:104AD000A6010E94D5020F900F900F900F900F909B
:104AE00080E090E01F910F91FF90EF90DF90CF90CA
:104AF000BF90AF909F908F9008950E94DA180E9407
:104B0000371880E090E0089560E0FC0183850C9404
:104B1000AB0E60E0FC0185810C94AB0E61E0FC0102
:104B200083850C94AB0E61E0FC0185810C94AB0E87
:104B3000CF93DF93FB01C68DD78D0E944732BE0114
:104B40000E94053280E090E0DF91CF910895CF93ED
:104B5000DF9380919F0B9091A00B892BF1F48CE354
:104B600090E00E945C48EC01FC01CC96118210821E
:104B70003C96E817F907D1F7198218821D861C8622
:104B8000198E188E1DA21CA219AA18AACE010E9465
:104B9000681BD093A00BC0939F0B80919F0B9091AB
:104BA000A00BDF91CF910895089508950895089579
:104BB0001F920F920FB60F9211240BB60F922F93E4
:104BC0003F934F935F936F937F938F939F93AF9395
:104BD000BF93EF93FF93E0914207F091430719953C
:104BE000FF91EF91BF91AF919F918F917F916F91C5
:104BF0005F914F913F912F910F900BBE0F900FBE81
:104C00000F901F901895CF93DF93EC01FC01E759AB
:104C1000FF4F1082379781E0808360E08D810E9492
:104C2000AB0E8F859889892B31F060E08B85DF9101
:104C3000CF910C94AB0EDF91CF910895CF93DF937A
:104C4000EC018B890E94830E2E8930E08217930736
:104C500011F48F8901C080E0DF91CF910895CF9347
:104C6000DF93EC0189890E94830E2E8930E0821740
:104C7000930711F48F8901C080E0DF91CF910895EF
:104C8000CF93DF93EC018DA5882311F061E001C083
:104C900060E08F810E94AB0E8EA5882329F08FA53E
:104CA000882311F061E001C060E08D85DF91CF9134
:104CB0000C94AB0ECF93DF93EC018DA5882311F0FC
:104CC00060E001C061E08F810E94AB0E8EA5882359
:104CD00029F08FA5882311F060E001C061E08D8587
:104CE000DF91CF910C94AB0ECF93DF93EC0161E099
:104CF00089850E94AB0E8EA5882321F061E08F8507
:104D00000E94AB0EC959DF4F1882DF91CF910895F1
:104D1000CF93DF93EC0160E089850E94AB0E8EA5F6
:104D2000882321F060E08F850E94AB0EC959DF4FC8
:104D300081E08883DF91CF910895CF92DF92EF9247
:104D4000FF920F931F93CF93DF93FC0142AF53AFBA
:104D500064AF75AFDC01DE964D935D936D937C93EC
:104D6000139714960D931D932D933C931397EC0179
:104D7000CA5BDF4FE88284A9882389F084A581116A
:104D800009C037FF0CC01D921D921D921C921397F3
:104D900081E006C01016110612061306A4F380E087
:104DA00045A956A967A970AD14161506160617066B
:104DB0003CF591AD992321F10D911D912D913C91DF
:104DC00013976801790137FF07C0CC24DD247601F1
:104DD000C01AD10AE20AF30A4C155D056E057F057B
:104DE0007CF437FF07C070956095509541955F4FF3
:104DF0006F4F7F4F4D935D936D937C93139781E03D
:104E0000DF01A15BBF4F1D921D921D921C92139753
:104E1000E15AFF4F91E09083DF91CF911F910F9165
:104E2000FF90EF90DF90CF9008950F931F93CF9353
:104E3000DF938C01D62FFC018589811109C0C8013F
:104E40000EDFC82FC801FADED11108C08C2F06C0B2
:104E5000C801F4DEC82FC80102DFF6CFDF91CF9181
:104E60001F910F910895CF93DF93EC01FC01E75957
:104E7000FF4F81E0808339978081B297882341F08A
:104E800080819181A281B3810196A11DB11D07C0CE
:104E900080819181A281B3810197A109B1098083A9
:104EA0009183A283B383FE01E459FF4F20813181B6
:104EB000DE01A659BF4FC9019595879520FD03C016
:104EC000ED91FC910DC0FE01E80FF91F0190F081FA
:104ED000E02D2D913C91E20FF31F0190F081E02D28
:104EE0008C0F9D1F19958F859889892B11F1FE01D3
:104EF000E059FF4F20813181DE01A259BF4FC90126
:104F00009595879520FD03C0ED91FC910DC0FE01A4
:104F1000E80FF91F0190F081E02D2D913C91E20FF7
:104F2000F31F0190F081E02D8C0F9D1FDF91CF9139
:104F30001994DF91CF9108958F929F92AF92BF9273
:104F4000CF92DF92EF92FF920F931F93CF93DF9355
:104F5000EC01FC01E15BFF4F6081718182819381F3
:104F60000E94074E6B017C0168A979A98AA99BA9B7
:104F70000E94094E9B01AC0160E074E284E799E471
:104F80000E94F74F4B015C01FE01E55AFF4F608123
:104F90007181828193810E94074E9B01AC01C50102
:104FA000B4010E94F74F4B015C018E010D5A1F4F57
:104FB00020E030E040E05FE30E94684E9B01AC01DE
:104FC000C701B6010E94934F0E946450F8016083AC
:104FD000718382839383C95ADF4FA5019401C7016E
:104FE000B6010E94934F0E946450688379838A833C
:104FF0009B83DF91CF911F910F91FF90EF90DF90F6
:10500000CF90BF90AF909F908F9008950F931F9374
:10501000CF93DF93FC01E759FF4F20812223B9F0A2
:105020007A970081118122813381389640815181A4
:1050300062817381041715072607370710F1EC0109
:10504000E2DDCE01DF91CF911F910F9175CFFC0171
:10505000E15AFF4F20812223A1F070970081118136
:10506000228133813496408151816281738104179A
:1050700015072607370728F0DF91CF911F910F9171
:10508000F2CEDF91CF911F910F9108952F923F9211
:105090004F925F926F927F928F929F92AF92BF9248
:1050A000CF92DF92EF92FF920F931F93CF93DF93F4
:1050B000CDB7DEB762970FB6F894DEBF0FBECDBF97
:1050C0008C017C0126E4E20EF11CD7018C91980141
:1050D000205A3F4FF801EF59FF4F6F01A801425C82
:1050E0005F4F4A0114971D01882341F0F80184A500
:1050F000D9018C9381E0F60180832FC0DA014D91B4
:105100005D916D917C91F10180819181A281B3814A
:10511000BB24B394481759076A077B070CF0B12CDE
:10512000F901B08277FF07C0709560955095419561
:105130005F4F6F4F7F4FB7FF07C0B095A095909519
:1051400081959F4FAF4FBF4F21E0481759076A071E
:105150007B070CF420E0D6012C93F40140815181AF
:1051600062817381411551056105710559F4F8019A
:10517000848D958DA68DB78DE55AFF4F80839183E1
:10518000A283B383F10180819181A281B381F8016F
:1051900042AC53AC64AC75AC9801215A3F4F5901F5
:1051A000481659066A067B0634F4481759076A07F9
:1051B0007B077CF00AC084159505A605B7052CF47D
:1051C00084179507A607B70724F0D7018C91882389
:1051D000D9F0F50180818823B9F0D7018C91811134
:1051E00005C0F701808181110FC006C060E0C801D1
:1051F0001CDE8111F6CF17C0D6016C9181E06827C3
:10520000C80113DE882379F0D5011C9260E0C80143
:105210000CDE882309F4C6C1F801FE9610821182C3
:1052200012821382BFC1D80194962D913D914D9168
:105230005C91979729833A834B835C8358962D9191
:105240003D914D915C915B972D833E834F835887B1
:105250005C962D913D914D915C915F9729873A879E
:105260004B875C87F10180819181A281B381F80134
:10527000FE96C080D180E280F380F80142AD53AD4C
:1052800064AD75ADED59FF4F108231961082380133
:10529000F5E66F0E711CF301108298012A593F4FF9
:1052A000F9011082329610824C015D01841A950A30
:1052B000A60AB70AB7FE08C0B094A0949094809450
:1052C000811C911CA11CB11C481759076A077B0758
:1052D0002CF4C41AD50AE60AF70A04C0C81AD90A77
:1052E000EA0AFB0AD501C401B595A795979587955C
:1052F0008D879E87AF87B88BD801A859BF4F1D01F6
:10530000F7FC05C08C149D04AE04BF044CF4F801F6
:1053100000A0F1A1E02DFA8BE98B81E0D9011BC03F
:105320002D853E854F8558892C153D054E055F0519
:1053300008F454C089819A81AB81BC818C159D058C
:10534000AE05BF0564F42D813E812F5F3F4F3A8B40
:10535000298B81E0D3018C93F10180839EC0C7012A
:10536000B6010E94094E2B013C0169817A818B8133
:105370009C810E94094E9B01AC01C301B2010E94B5
:10538000F74F2B013C016D817E818F8198852985A6
:105390003A854B855C85621B730B840B950B0E94D1
:1053A000094E9B01AC01C301B2010E94684E2B0162
:1053B0003C0169857A858B859C850E94094E9B01FD
:1053C000AC01C301B2010E94934F0E945F507A8BDF
:1053D000698B81E0F801ED59FF4F5CC0D501C40134
:1053E00029813A814B815C81821B930BA40BB50B05
:1053F000C816D906EA06FB065CF42D813E812E5FB5
:105400003F4F3A8B298B81E0F801EB59FF4F42C0A7
:10541000C501B4016C197D098E099F090E94094ECE
:105420002B013C0169817A818B819C810E94094E0C
:105430009B01AC01C301B2010E94F74F2B013C015B
:105440006D817E818F81988529853A854B855C8524
:10545000621B730B840B950B0E94094E9B01AC01E0
:10546000C301B2010E94684E2B013C0169857A8517
:105470008B859C850E94094E9B01AC01C301B20142
:105480000E94934F0E945F507A8B698B81E0F801F4
:10549000EC59FF4F8083D1018C93F80184818823DC
:1054A000B1F00E941E10D80112964D905C90139797
:1054B000052C000C66087708DC01CB0184199509DE
:1054C000A609B709893E9340A105B10568F4F80122
:1054D000E55AFF4F29893A89C901A0E0B0E08083ED
:1054E0009183A283B38392CE0E941E10D80113969B
:1054F0007C936E93129784E294E00E94E53B81EBEB
:1055000095E00E94E53B60E070E0CB010E94313CF9
:1055100087EB95E00E94E53BC701B6010E94313C54
:105520008DEB95E00E94E53BC501B4010E94313C42
:1055300083EC95E00E94E53B4AE06D857E858F8592
:1055400098890E94E63B8AEC95E00E94E53B6981E0
:105550007A818B819C810E94313C80ED95E00E9494
:10556000E53B69857A858B859C850E94313C86ED7B
:1055700095E00E94E53B6D817E818F8198850E9438
:10558000313C8CED95E00E94E53B8EE496E00E9474
:10559000E53B89899A890E94583C8CE993E00E94F6
:1055A000E53B95CF62960FB6F894DEBF0FBECDBF38
:1055B000DF91CF911F910F91FF90EF90DF90CF90EF
:1055C000BF90AF909F908F907F906F905F904F9023
:1055D0003F902F9008950F931F93FC01EA5BFF4FBC
:1055E0002081211110C038970081118122813381DF
:1055F0003496408151816281738104171507260713
:10560000370744F404C0FC0124A5222319F01F919C
:105610000F9150CB1F910F9133CBFC01138212825B
:1056200014821682158210861782128611861486BD
:10563000138616861586108A1786128A118A148A8E
:10564000138ADC01A15ABF4F1C9212AE13AE14AEE6
:1056500015AE91971D921D921D921C921397149650
:105660001D921D921D921C92139714961C925A968D
:105670001C9211961C9212961C9211961C921196D5
:105680001C9211961C9211961C9211961C921196C6
:105690001C92119683E995E211969C938E93129633
:1056A00011961C921E9212968EE895E211969C938A
:1056B0008E93129611961C921E92129689E895E28C
:1056C00011969C938E93129611961C921E9212968E
:1056D00084E895E28D939C93E858FF4F11821082E5
:1056E000089508956E3471050CF050C06B34710547
:1056F0000CF08FC06C32710554F5693271050CF0F5
:1057000088C06831710594F46F3071050CF081C068
:105710006630710544F4623071050CF07AC0672B75
:1057200009F075C076C06B5071096EC062327105A8
:105730003CF46F3171050CF06CC06951710964C0A3
:10574000645271096230710508F061C062C06A3349
:1057500071057CF4673371050CF05BC06D32710527
:105760000CF455C0603371050CF453C063537109D8
:105770004BC0643471053CF4613471050CF049C0D0
:105780006D53710941C0675471093EC06638710597
:10579000F4F463387105ECF56237710564F46F3623
:1057A0007105BCF56536710594F1683671058CF1AB
:1057B0006956710929C06C37710534F46937710570
:1057C00044F56357710920C06D5771091DC0603DD4
:1057D00071057CF46D3C7105E4F46439710534F4B1
:1057E00061397105B4F46D5871090EC0695C7109B5
:1057F0000BC06A3D710534F4673D710554F4635D77
:10580000710902C06D5D71096330710510F080E0AF
:10581000089581E00895603E710508F0D8C3FB014A
:105820008827EC57FF4F8F4F0C94B35081E090E0E6
:10583000A0E0B0E08093560790935707A0935807D5
:10584000B0935907089510925A0710925B0710926F
:105850005C0710925D07089510925E0710925F0733
:105860001092600710926107089581E090E0A0E037
:10587000B0E08093620790936307A0936407B093AE
:1058800065070895109266071092670710926807DF
:1058900010926907089583E090E0A0E0B0E0809363
:1058A0006A0790936B07A0936C07B0936D070895F8
:1058B00088E790E0A0E0B0E08093820790938307B0
:1058C000A0938407B0938507089588E790E0A0E04F
:1058D000B0E08093860790938707A0938807B093E2
:1058E0008907089588E790E0A0E0B0E080938A07F8
:1058F00090938B07A0938C07B0938D070895109217
:1059000092071092930710929407109295070895AA
:105910001092960710929707109298071092990785
:10592000089581E090E0A0E0B0E080939A07909322
:105930009B07A0939C07B0939D07089510929E0724
:1059400010929F071092A0071092A107089510923D
:10595000A2071092A3071092A4071092A50708951A
:105960001092A6071092A7071092A8071092A907F5
:1059700008951092AA071092AB071092AC071092EC
:10598000AD0708951092AE071092AF071092B007BE
:105990001092B10708951092B2071092B3071092B7
:1059A000B4071092B50708951092BA071092BB077A
:1059B0001092BC071092BD0708951092BE07109276
:1059C000BF071092C0071092C10708951092C20736
:1059D0001092C3071092C4071092C5070895109241
:1059E000D2071092D3071092D4071092D5070895CA
:1059F0001092D6071092D7071092D8071092D907A5
:105A000008951092DA071092DB071092DC071092CB
:105A1000DD07089581E090E0A0E0B0E08093E60724
:105A20009093E707A093E807B093E907089581E012
:105A300090E0A0E0B0E08093EA079093EB07A0939A
:105A4000EC07B093ED0708958CE291E0A0E0B0E0A0
:105A50008093FA079093FB07A093FC07B093FD0790
:105A600008958CE291E0A0E0B0E08093FE0790936F
:105A7000FF07A0930008B093010808958CE291E01D
:105A8000A0E0B0E08093020890930308A09304087C
:105A9000B0930508089510920A0810920B0810920E
:105AA0000C0810920D08089510920E0810920F081D
:105AB0001092100810921108089510921208109276
:105AC00013081092140810921508089510922208D5
:105AD000109223081092240810922508089510921D
:105AE0002608109227081092280810922908089575
:105AF00081E090E0A0E0B0E080932A0890932B082A
:105B0000A0932C08B0932D08089585E090E0A0E0C4
:105B1000B0E08093320890933308A0933408B09398
:105B20003508089585E090E0A0E0B0E08093360865
:105B300090933708A0933808B0933908089589E105
:105B400090E0A0E0B0E080933A0890933B08A093E7
:105B50003C08B0933D08089582E390E0A0E0B0E0F7
:105B600080934A0890934B08A0934C08B0934D083B
:105B7000089582E390E0A0E0B0E080934E08909317
:105B80004F08A0935008B0935108089582E390E025
:105B9000A0E0B0E08093520890935308A09354087B
:105BA000B0935508089582E390E0A0E0B0E08093C0
:105BB0005A0890935B08A0935C08B0935D08089521
:105BC00082E390E0A0E0B0E080935E0890935F08ED
:105BD000A0936008B0936108089582E390E0A0E08C
:105BE000B0E08093620890936308A0936408B09338
:105BF0006508089580E991E0A0E0B0E08093720824
:105C000090937308A0937408B0937508089580E981
:105C100091E0A0E0B0E08093760890937708A0939D
:105C20007808B0937908089580E991E0A0E0B0E0A9
:105C300080937A0890937B08A0937C08B0937D08AA
:105C4000089510928208109283081092840810928E
:105C50008508089510928608109287081092880887
:105C600010928908089510928A0810928B08109259
:105C70008C0810928D08089510929A0910929B0931
:105C800010929C0910929D09089510929E091092FD
:105C90009F091092A0091092A10908951092A209DB
:105CA0001092A3091092A4091092A50908951092C8
:105CB000EA081092EB081092EC081092ED08089593
:105CC0001092EE081092EF081092F0081092F1086E
:105CD00008951092F2081092F3081092F4081092AE
:105CE000F50808951092FA081092FB081092FC082B
:105CF0001092FD0808951092FE081092FF0810926D
:105D000000091092010908951092020910920309E6
:105D10001092040910920509089585E090E0A0E032
:105D2000B0E08093120990931309A0931409B093E3
:105D30001509089585E090E0A0E0B0E08093160991
:105D400090931709A0931809B0931909089585E055
:105D500090E0A0E0B0E080931A0990931B09A09313
:105D60001C09B0931D09089584EB95E1A0E0B0E013
:105D70008093220990932309A0932409B0932509C5
:105D8000089584EB95E1A0E0B0E08093260990931C
:105D90002709A0932809B0932909089584EB95E178
:105DA000A0E0B0E080932A0990932B09A0932C09DE
:105DB000B0932D09089585E090E0A0E0B0E08093D5
:105DC0003A0990933B09A0933C09B0933D0908958B
:105DD00085E090E0A0E0B0E080933E0990933F0919
:105DE000A0934009B0934109089585E090E0A0E0B8
:105DF000B0E08093420990934309A0934409B09383
:105E00004509089510924A0910924B0910924C09C5
:105E100010924D09089510924E0910924F09109258
:105E20005009109251090895109252091092530985
:105E30001092540910925509089510926209109217
:105E40006309109264091092650908951092660919
:105E500010926709109268091092690908951092CA
:105E60006A0910926B0910926C0910926D090895DD
:105E700010927A0A10927B0A10927C0A10927D0A84
:105E800008958CE390E0A0E0B0E080937E0A9093C8
:105E90007F0AA093800AB093810A089581E090E080
:105EA000A0E0B0E08093820A9093830AA093840AD2
:105EB000B093850A089510928A0A10928B0A109264
:105EC0008C0A10928D0A08958CE390E0A0E0B0E077
:105ED00080938E0A90938F0AA093900AB093910AB0
:105EE000089581E090E0A0E0B0E08093920A909362
:105EF000930AA093940AB093950A08951092A20A67
:105F00001092A30A1092A40A1092A50A08958CE395
:105F100090E0A0E0B0E08093A60A9093A70AA09337
:105F2000A80AB093A90A089581E090E0A0E0B0E04B
:105F30008093AA0A9093AB0AA093AC0AB093AD0ADF
:105F400008951092B20A1092B30A1092B40A1092F5
:105F5000B50A08958CE390E0A0E0B0E08093B60A23
:105F60009093B70AA093B80AB093B90A089581E054
:105F700090E0A0E0B0E08093BA0A9093BB0AA093AF
:105F8000BC0AB093BD0A08951092CA0A1092CB0AB7
:105F90001092CC0A1092CD0A08958CE390E0A0E014
:105FA000B0E08093CE0A9093CF0AA093D00AB0932A
:105FB000D10A089581E090E0A0E0B0E08093D20A99
:105FC0009093D30AA093D40AB093D50A0895660F8C
:105FD000771F660F771FFB01EA5AF84F1082118274
:105FE0001282138208950F931F93CF93DF938C0136
:105FF000C0E0D0E0BE01C80175DB882319F0BE0106
:10600000C80109DC2196C13ED105A1F7DF91CF91EE
:106010001F910F9108954F925F926F927F928F928E
:106020009F92AF92BF92CF92DF92EF92FF92CF9367
:10603000DF935B01EB01CC0FDD1FCE010E941F4FF0
:10604000482E512C612C712CCE0101960E941F4FBD
:10605000C82ED12CE12CF12C8DE8A81AB10883E0D0
:10606000A816B10488F5CE0144960E941F4F882ED1
:10607000912CA12CB12CCE0145960E941F4F482F88
:1060800050E060E070E08FEF88169104A104B10445
:10609000A9F44F3F51056105710581F48FEF481652
:1060A00051046104710481F48FEFC816D104E10436
:1060B000F10451F46FEF7FEFCB012BC04038510555
:1060C000610571056CF0F6CF80E8C816D104E104D3
:1060D000F10484F740E050E0BA01812C912C540186
:1060E000FE2CED2CDC2CCC24C40CD51CE61CF71C9F
:1060F000540199248824C80CD91CEA1CFB1C742F59
:10610000662755274427CB01BA016C0D7D1D8E1DD6
:106110009F1DDF91CF91FF90EF90DF90CF90BF90C8
:10612000AF909F908F907F906F905F904F90089569
:106130000C94F1480C94F1480C94F148CF93DF9300
:10614000EB0120E030E040E85FE36A817B818C81F5
:106150009D810E94034E811113C082EE95E00E9442
:10616000E53B0E942E17FC01E25BFF4F108211827B
:1061700012821382E05DFE4F108A118A128A138AFE
:1061800020E030E040E85FE36E817F81888599857B
:106190000E94034E811113C082EF95E00E94E53BFF
:1061A0000E942E17FC01E853FF4F108211821282C9
:1061B0001382EC52FF4F108A118A128A138A20E050
:1061C00030E040E85FE36A857B858C859D850E9491
:1061D000034E811113C082E096E00E94E53B0E94CD
:1061E0002E17FC01EE5BFE4F108211821282138289
:1061F000E858FF4F108A118A128A138A0E94DA180F
:106200000E94E41780E090E0DF91CF9108950F9312
:10621000CF93DF938091A30B811173C081E08093B2
:10622000A30B0E942E17EC0106B126B1409100018C
:10623000609100010295017026FB222720F9417030
:106240006695617082589E4F25D506B126B140B142
:1062500060B1017022FB222720F943FB442740F95B
:1062600066956170CE0184569E4F14D502B322B359
:1062700040B160B1017022FB222720F9441F44275E
:10628000441F65FB662760F9CE0186549E4F02D5F8
:10629000FE01E159FF4F8081882361F07097808172
:1062A0009181A281B3810196A11DB11D808391834B
:1062B000A283B383FE01E751FF4F8081882361F001
:1062C000709780819181A281B3810196A11DB11D3A
:1062D00080839183A283B383FE01ED59FE4F8081B9
:1062E000882369F0CD5ADE4F88819981AA81BB81CC
:1062F0000196A11DB11D88839983AA83BB83109247
:10630000A30BDF91CF910F9108958F929F92AF923F
:10631000BF92CF92DF92EF92FF920F931F930E9452
:106320002E1721E02F931F921F921F921F92812CF4
:10633000912CA12CB12CC12CD12C76019701860176
:10634000B701A6010E94D5020F900F900F900F90F9
:106350000F9080E090E01F910F91FF90EF90DF9001
:10636000CF90BF90AF909F908F900895EF92FF9243
:106370000F931F93CF93DF9300D01F92CDB7DEB75B
:106380008B017B01EE0CFF1C622FC70129833A832E
:106390004B835C830E94274F29813A814B815C812A
:1063A000992757FD9A95852F742F632FC701019662
:1063B0000E94274F0D58110929813A814B815C8138
:1063C00003301105A8F4BA01992777FD9095892F1C
:1063D000C70144960E94274F29813A814B815C81F5
:1063E000652F772788279927C70145960E94274F51
:1063F00080E090E00F900F900F900F90DF91CF9181
:106400001F910F91FF90EF900895CF92DF92EF923E
:10641000FF92CF93DF93EB0165D9882359F1FE01F9
:10642000EE0FFF1FEE0FFF1FEA5AF84FC080D1801A
:10643000E280F38082E196E00E94E53B8EE496E004
:106440000E94E53B86E196E00E94E53BCE010E947A
:10645000583C8EE496E00E94E53B88E196E00E947D
:10646000E53BC701B6010E94313C0E94DA180E9448
:10647000E41704C08AE196E00E94E53B80E090E0EA
:10648000DF91CF91FF90EF90DF90CF900895EF9242
:10649000FF920F931F93CF93DF938091A40B909162
:1064A000A50B892B09F064C084E090E00E945C4851
:1064B000EC0160E070E0AFDD16161706F4F0CE01D7
:1064C00092DD96E5E92E97E0F92E00E010E0B801A4
:1064D000CE0108D9882341F0F70120813181428122
:1064E0005381B801CE0142DF0F5F1F4FF4E0EF0E82
:1064F000F11C0639110559F737C063E070E0CE0191
:106500008ADD613071058105910561F586E5E82E2A
:1065100087E0F82E00E010E0B801CE01E3D8882330
:10652000C1F0B801CE0177DDF7016083718382830A
:1065300093836F3F7F4F8F4F9F4F59F4B801CE0128
:106540006AD9F7012081318142815381B801CE019E
:106550000DDF0F5F1F4FF4E0EF0EF11C013E110540
:10656000D9F602C0CE013FDDD093A50BC093A40B9A
:106570008091A40B9091A50BDF91CF911F910F916A
:10658000FF90EF9008950895089508958091A10BCC
:106590009091A20B892B41F481E090E00E945C482D
:1065A0009093A20B8093A10B8091A10B9091A20BD1
:1065B0000895EF92FF920F931F93CF93DF93162FBF
:1065C000072F7A014115510559F4862F0E94830E39
:1065D00031E020E0019709F030E0C32FD22F26C030
:1065E0004130510509F5262F663310F02AEC260FAD
:1065F00080917B00922F9870877F892B80937B00FE
:106600002770206420937C0080917A0080648093BE
:106610007A0080917A0086FDFCCFC091780080914D
:106620007900D0E0D82B02C0C0E0D0E082E0E816CC
:10663000F10410F58CE396E00E94E53B8EE496E0D1
:106640000E94E53B86E196E00E94E53B812F902F7A
:106650000E94583C8EE496E00E94E53B88E196E07B
:106660000E94E53BCE010E94583C0E94DA180E942D
:10667000E41780E090E002C081E090E0DF91CF91EC
:106680001F910F91FF90EF90089580E496E00E9493
:10669000E53B0E94DA180E94211B0E94DA180E9432
:1066A000F6171DD240E050E068E070E082DF17D2BC
:1066B00040E050E069E070E07CDF11D240E050E063
:1066C0006AE070E076DF0BD240E050E06DE070E011
:1066D00070DF80E090E008950F931F93CF93DF93D6
:1066E0008B01EA01AB01415051094433510508F0D7
:1066F000D4C02230310508F0D0C048E3429FF001F9
:10670000439FF00D1124E60FF71FE80FF91F81E0FA
:106710008083232B11F46C2F07C061E0802F0E942F
:106720009F0F209739F460E0802F0E94AB0E80E02D
:1067300090E0B5C0CF3FD10509F4ADC0F801EF5DE1
:10674000FB4FE4918E2F90E0FC013197E231F1058F
:1067500008F09DC08827EC59FE4F8F4F0C94B35022
:1067600084B5806884BDC7BDE2CF84B5806284BD36
:10677000C8BDDDCF80918000806880938000D09379
:106780008900C0938800D3CF80918000806280937D
:106790008000D0938B00C0938A00C9CF8091800085
:1067A000886080938000D0938D00C0938C00BFCF11
:1067B0008091B00080688093B000C093B300B7CFE1
:1067C0008091B00080628093B000C093B400AFCFDE
:1067D00080919000806880939000D0939900C0933E
:1067E0009800A5CF80919000806280939000D09314
:1067F0009B00C0939A009BCF80919000886080930B
:106800009000D0939D00C0939C0091CF8091A000F8
:1068100080688093A0008091A0008F7B8093A0006F
:10682000D093A900C093A80082CF8091A00080627D
:106830008093A000D093AB00C093AA0078CF809142
:10684000A00088608093A000D093AD00C093AC00FE
:106850006ECF80912001806880932001D093290120
:10686000C093280164CF8091200180628093200131
:10687000D0932B01C0932A015ACF809120018860C8
:1068800080932001D0932D01C0932C0150CFC038AC
:10689000D1050CF448CF61E047CF81E090E0DF9173
:1068A000CF911F910F9108950C94F1480C94F148E9
:1068B0000C94F1480C94F1480C94F1480C94F14874
:1068C0000C94F1480C94F1480C94F1480C94F14864
:1068D0000C94F1488F929F92AF92BF92CF92DF9229
:1068E000EF92FF920F931F930E942E1760E070E0CB
:1068F0004ED2892BD1F40E942E171F921F9221E0B5
:106900002F931F921F92812C912CA12CB12CC12C62
:10691000D12C760197018601B701A6010E94D5020C
:106920000F900F900F900F900F9080E090E01F91CC
:106930000F91FF90EF90DF90CF90BF90AF909F901E
:106940008F9008958F929F92AF92BF92CF92DF92D5
:10695000EF92FF920F931F930E942E1761E070E059
:1069600016D2892BD1F40E942E171F9221E02F936B
:106970001F921F921F92812C912CA12CB12CC12C03
:10698000D12C760197018601B701A6010E94D5029C
:106990000F900F900F900F900F9080E090E01F915C
:1069A0000F91FF90EF90DF90CF90BF90AF909F90AE
:1069B0008F900895EF92FF920F931F93CF93DF93E1
:1069C00000D01F92CDB7DEB7FB0122A133A144A1B5
:1069D00055A1068D178D29833A834B835C8357DD40
:1069E0007C01FC018281938129813A814B815C8108
:1069F0008F30F7E29F072CF40196F701938382838F
:106A000003C0F70113821282B801C70129833A83B8
:106A10004B835C830E94722B29813A814B815C817C
:106A2000882391F0F801EE0FFF1FEE0FFF1FEA5AC7
:106A3000F84F2083318342835383B801C70196DC2A
:106A4000B801C701E2DC03C08AE196E0BED60E942D
:106A5000A7250E94681B80E090E00F900F900F9098
:106A60000F90DF91CF911F910F91FF90EF900895BC
:106A70000F931F93CF93DF930ADD8C01C0E0D0E02A
:106A8000BE01C8010E94722B882319F0BE01C80103
:106A9000BCDC2196C13ED10599F787E496E095D6F6
:106AA0000E94DA180E94E41780E090E0DF91CF9115
:106AB0001F910F9108958BE496E087D685E593E0CA
:106AC00084D60E94DA180E94E41780E090E00895CE
:106AD0000E94DA18FC01148680E090E0089580910D
:106AE000A60B9091A70B892BA1F480E790E00E9460
:106AF0005C48FC01F9969C0123593F4FDF01D89770
:106B00001C921192E217F307C9F79093A70B809399
:106B1000A60B8091A60B9091A70B08956F927F9280
:106B20008F929F92AF92BF92CF92DF92EF92FF929D
:106B30000F931F93CF93DF93FB01E2A8F3A886A4E2
:106B400097A4A0A8B1A8C6A0D7A062A073A0068DE4
:106B5000178DC5DFEC019701A301B801BDDDC501AB
:106B6000B4010E94E60F9701A601B801CE01B4DD81
:106B700080E090E0DF91CF911F910F91FF90EF9017
:106B8000DF90CF90BF90AF909F908F907F906F904D
:106B900008950F931F93CF93DF93FB0102A913A9CD
:106BA000C68DD78D9CDFA801BE0103DD80E090E09B
:106BB000DF91CF911F910F9108951F93CF93DF9392
:106BC0001F92CDB7DEB7FB0162A9168D698387DFFF
:106BD0006981812F0E949F0F80E090E00F90DF91EC
:106BE000CF911F910895EF92FF920F931F93CF9330
:106BF000DF93FB01E2A8F3A802A113A1C68DD78DF4
:106C00006EDF9701A801BE0167DD80E090E0DF91B3
:106C1000CF911F910F91FF90EF90089508950895DF
:106C2000089508950895CF93DF93EC0188810E9421
:106C3000830E21E0892B09F420E02C878C810E94AF
:106C4000830E21E0892B09F420E02E87888D998D11
:106C50000197D1F48A810E94830E21E0892B09F4E7
:106C600020E02D878E810E94830E21E0892B09F47C
:106C700020E02F879C858D85981749F08E85821797
:106C800031F09A878B8703C08C858A872B87DF91A9
:106C9000CF9108950F93FC0192859087838581871A
:106CA000A08DB18D119721F4621721F0401711F0DA
:106CB0006287438783858823D1F0828591110AC03A
:106CC0008823A9F080899189A289B3890197A109B4
:106CD000B10909C081110BC080899189A289B3894A
:106CE0000196A11DB11D808B918BA28BB38B0F914F
:106CF0000895CF93DF93FC0124893589468957890C
:106D0000C28DD38D60897189828993892031E7E2B0
:106D10003E074105510529F0121613061406150603
:106D200024F0DE019B01AC0109C00E94985020E1D3
:106D300037E240E050E00E94354FDE010E945B4F99
:106D4000DF91CF910895FC0181E090E0958F848FD1
:106D50001182108215821482108A118A128A138A73
:106D6000118E108E80E197E2A0E0B0E0848B958BCD
:106D7000A68BB78B12861086148615861686178604
:106D800008950895089508950895089508952F92F7
:106D90003F924F925F926F927F928F929F92AF92AB
:106DA000BF92CF92DF92EF92FF920F931F93CF93F8
:106DB000DF93CDB7DEB7A3970FB6F894DEBF0FBE53
:106DC000CDBF9BA38AA31B010E948A1D8AA19BA100
:106DD0000E949D1B8AA19BA10E9487138AA19BA14F
:106DE0000E94891321E022163104C9F132E02316F2
:106DF000310409F466C02114310409F095C0AAA039
:106E0000BBA040E1A40EB11C8AA19BA182589E4F59
:106E10009E838D83EAA1FBA1E45BFD4F90819B875C
:106E2000AAA1BBA1A359BD4FB887AF83EAA1FBA11B
:106E3000E956FD4FFF87EE872AA13BA127553D4F1D
:106E40003B8B2A8B4AA15BA147515E4F5A874987EA
:106E50008DE890E0998B888BA5E1B0E062C0AAA094
:106E6000BBA0BAE8AB0EB11CEAA1FBA1E456FE4FF1
:106E7000FE83ED83EAA1FBA1E35BFD4F20812B871D
:106E80004AA15BA14F585D4F58874F838AA19BA1B0
:106E900087569D4F9F878E87AAA1BBA1A655BD4F40
:106EA000BB8BAA8BEAA1FBA1E551FE4FFA87E987CC
:106EB0002EE830E0398B288B46E150E05C834B8331
:106EC00036C0AAA0BBA05CEFA51A5EEFB50A8AA1E6
:106ED0009BA186549E4F9E838D83EAA1FBA1E25B1A
:106EE000FD4F90819B87AAA1BBA1AB58BD4FB8872E
:106EF000AF83EAA1FBA1E556FD4FFF87EE872AA1EC
:106F00003BA125553D4F3B8B2A8B4AA15BA14351A9
:106F10005E4F5A8749878FE890E0998B888BA7E16D
:106F2000B0E0BC83AB8303C080E596E00CC0C50134
:106F30000E942F26811105C0C5010E941E268823AC
:106F400069F081EE96E041D40E94DA1881E090E089
:106F5000909345078093440790E0D4C384E294E083
:106F600034D48FE796E031D4D5018C916FD487E18A
:106F700097E02BD48CE993E028D481E090E0E98578
:106F8000FA859183808341E050E0B5018AA19BA1FD
:106F90000E943219C5010E948826D5019C968C91C9
:106FA0008501005A1F4F882339F0C5010E945A26D7
:106FB00081E0F801808305C0C5010E944026D80108
:106FC0001C928D819E8195DEF501FE966083718312
:106FD00082839383EF81F88510821182128213825B
:106FE000EAA1FBA1E359FD4F1082118212821382A4
:106FF000EAA1FBA1EF58FD4F108211821282138289
:10700000EAA1FBA1EB58FD4F10821182128213827C
:1070100086E090E0A985BA858D939C9346E050E088
:10702000B5018AA19BA10E94321941E050E0B5014F
:107030008AA19BA10E941719412C512C3201439423
:107040008AA19BA1820D931DFC01E755FD4FFD8791
:10705000EC874101880C991C880C991CC40183564B
:107060009D4F2AA13BA1280F391F3D8B2C8BC101BD
:10707000815A9E4F880F991F4AA15BA1480F591F43
:10708000598F488FC40185579D4FAAA1BBA1A80F56
:10709000B91FBB8FAA8FF401E158FD4FFD8FEC8F14
:1070A0008AA19BA1880D991D9C012A5E3D4F3F8FAF
:1070B0002E8FAC85BD858C918823B1F0A4014359F6
:1070C0005D4FEAA1FBA14E0F5F1FCC88DD88E88CE5
:1070D000F98C0A8D1B8D2C8D3D8D2E0F3F1F6D81E0
:1070E0007E81C5010E94CB1288EA9BE00E948E0B34
:1070F0001816190624F01A82198210E01DC088EAB9
:107100009BE00E946C0B8F7D85349105A1F78DE982
:1071100094E05BD30E94DA1821E0DC011C962C93EA
:1071200082E693E052D30E94DA180E94E417E1E06D
:10713000F0E0FA83E98311E0C5010E942F26811156
:10714000D0C2C5010E941E268111CBC21111C9C235
:10715000AE85BF856D917C91072E000C880B990B35
:107160000E94094E9B01AC01EF81F885608171811D
:10717000828193810E94034E87FFB3C2C5010E94A2
:1071800033278AA19BA1880D991D8C010A5E1D4F92
:10719000F801208131814281538160E573EC80E008
:1071A00090E00E94354FC9010E94DB0FD8012D915C
:1071B0003D914D915C91A3E0B0E00E94514F9B0145
:1071C000AC01C301B2010E94354F672B682B692BBC
:1071D00039F48EE593E0F9D20E94DA180E94E417A0
:1071E000C5010E940326AE8DBF8D2D913D914D911D
:1071F0005C9160E573EC80E090E00E94354FC9013E
:107200000E94DB0FBFEF4B1A5B0A6B0A7B0AE98116
:10721000FA81EF2B09F44DCF21E030E03A83298346
:1072200042E050E0B5018AA19BA10E94171984E2B7
:1072300094E0CBD28FE796E0C8D2D5018C9106D3EB
:1072400086E896E0C2D28CE993E0BFD2E981FA8168
:10725000EF2BD1F489E996E0B8D28EE496E0B5D26E
:1072600086E196E0B2D28B819C8122D38EE496E0B7
:10727000ACD288E196E0A9D2FB858F2F90E018D39D
:107280000E94DA180E94E4178AA19BA10E9487132A
:107290008AA19BA10E94891384E294E096D28FE791
:1072A00096E093D2D5018C91D1D28DE996E08DD222
:1072B0008CE993E08AD2EF81F885108211821282E4
:1072C0001382D5019C968C918501005A1F4F88230B
:1072D00031F0C5010E944026F801108206C0C501A8
:1072E0000E945A2681E0D8018C938D819E8101DD18
:1072F000F501FE966083718382839383EAA1FBA1EB
:10730000E359FD4F1082118212821382EAA1FBA180
:10731000EF58FD4F1082118212821382EAA1FBA165
:10732000EB58FD4F10821182128213828D819E8153
:10733000E0DC6C8B7D8B8E8B9F8B412C512C320132
:1073400043948AA19BA1820D931DFC01E755FD4F3B
:10735000F98FE88F9101220F331F220F331F3C83D7
:107360002B83C90183569D4F4AA15BA1480F591F2A
:107370005B8F4A8FC101815A9E4F880F991FAAA126
:10738000BBA1A80FB91FBD8FAC8FC90185579D4FF9
:10739000EAA1FBA1E80FF91FFF8FEE8FC9012AA117
:1073A0003BA1820F931FAC014A5E5D4F59A348A3D6
:1073B000F2013197FD87EC874F0129813A81232B18
:1073C00009F0CFC0A88DB98D8C918823C9F02B818D
:1073D0003C8121583D4FEAA1FBA12E0F3F1F4B815D
:1073E0005C8143595D4F4E0F5F1FCA8CDB8CEC8C68
:1073F000FD8C0E8D1F8D6D817E81C5010E94CB128B
:1074000088EA9BE00E948E0B1816190614F010E013
:107410001DC088EA9BE00E946C0B8F7D853491052E
:10742000B1F78DE994E0D1D10E94DA1821E0DC01B6
:107430001C962C9382E693E0C8D10E94DA180E9431
:10744000E417E1E0F0E0FA83E98311E02C853D8563
:107450002A30310538F4AF81B8851D921D921D92F6
:107460001C921397BB85C501B11147C10E941E260E
:10747000811173C0112319F08C849D846EC0EE8538
:10748000FF8560817181072E000C880B990B0E948B
:10749000094E9B01AC01AF81B8856D917D918D91B5
:1074A0009C910E94034E87FFE7CFC5010E943327BE
:1074B0008B809C80EAA1FBA18E0E9F1EFAEE8F1A94
:1074C000FDEF9F0AD4012D913D914D915C9160E5B6
:1074D00073EC80E090E00E94354FC9010E94DB0F01
:1074E000F4012081318142815381A3E0B0E00E9408
:1074F000514F9B01AC01C301B2010E94354F672B74
:10750000682B692B91F48EE593E05FD10E94DA1825
:107510000E94E41784E294E058D181EB96E055D1C3
:10752000C201C6D18CE993E050D1C5010E94032667
:10753000A8A1B9A12D913D914D915C9160E573ECAD
:1075400080E090E00E94354FC9010E94DB0FBFEF41
:107550004B1A5B0A6B0A7B0A2BCF8FEB96E035D177
:1075600004C041E050E05A83498384E294E02DD185
:107570008FE796E02AD1D5018C9168D183ED96E012
:1075800024D18CE993E021D18D819E81B2DBEA89FF
:10759000FB89EF2BA1F0DC01CB012C893D894E89C1
:1075A0005F89821B930BA40BB50BB7FF07C0B09587
:1075B000A095909581959F4FAF4FBF4F4C0149814A
:1075C0005A81452BF9F489E996E0FFD08EE496E0E4
:1075D000FCD086E196E0F9D08889998969D18EE45A
:1075E00096E0F3D088E196E0F0D0B401092C000CCD
:1075F000880B990B0E94094E42E05FD10E94DA1875
:107600000E94E41785E090E0A985BA858D939C934C
:1076100045E050E0B5018AA19BA10E943219C50145
:107620000E9474268AA19BA10E9487138AA19BA114
:107630000E948913B1E02B163104A9F0E2E02E1666
:10764000310401F1232861F50E94DA18C401990C74
:10765000AA0BBB0B80934A0790934B07A0934C0750
:10766000B0934D071DC00E94DA18C401990CAA0BF3
:10767000BB0B80934E0790934F07A0935007B09396
:1076800051070EC00E94DA18C401990CAA0BBB0B5B
:107690008093520790935307A0935407B0935507D4
:1076A0000E94DA180E943718A985BA851D921C928B
:1076B00040E050E0B5018AA19BA10E94321940E050
:1076C00050E0B5018AA19BA10E9417190E94DA1807
:1076D000E981FA81F0934507E093440789819A8113
:1076E00011C08FEB96E071D0C5010E941E26882341
:1076F00009F496CDB1E0BB8793CD0E942F2681116E
:10770000BBCEB8CEA3960FB6F894DEBF0FBECDBFEA
:10771000DF91CF911F910F91FF90EF90DF90CF906D
:10772000BF90AF909F908F907F906F905F904F90A1
:107730003F902F900895CF93DF93FC01E452FE4FCA
:10774000408151814115510559F1EC01C052DE4F84
:107750002881398188529E4F24173507C8F4FC01CF
:1077600080819181009761F0FC01E20FF31F80811D
:107770008A3041F08D3029F48CE993E026D002C0A4
:1077800080E064D08881998101969983888308C0BC
:1077900040E050E06EE973E00E94E60D1982188225
:1077A000DF91CF910895009769F0FC0101900020CE
:1077B000E9F73197AF01481B590BBC0188EA9BE000
:1077C0000C942E0B80E090E00895EDCF8F929F9265
:1077D000AF92BF920F931F93CF93DF93CDB7DEB7D6
:1077E000A1970FB6F894DEBF0FBECDBF19A24230ED
:1077F00008F44AE08E010F5D1F4F842E912CA12CBE
:10780000B12CA50194010E94614FE62FB901CA0174
:1078100001501109EA3014F4E05D01C0E95CD801BF
:10782000EC93232B242B252B61F7C801BCDFA196F9
:107830000FB6F894DEBF0FBECDBFDF91CF911F9181
:107840000F91BF90AF909F908F900895E091A80BFB
:10785000F091A90B0190F081E02D682F88EA9BE060
:107860001994CF92DF92EF92FF92CF93DF9397FF1D
:1078700017C06B017C018DE2E9DFEC0166277727F9
:10788000CB016C197D098E099F094AE09FDF8C0F9F
:107890009D1FDF91CF91FF90EF90DF90CF900895E3
:1078A0004AE0DF91CF91FF90EF90DF90CF908ECFA5
:1078B000BC01990F880B990BD4CF4F925F926F92B6
:1078C0007F928F929F92AF92BF92CF92DF92EF9270
:1078D000FF926B017C01B42E9B01AC010E9494507D
:1078E000882319F086E397E027C026013701E89442
:1078F00077F82FEF3FEF4FE75FE7C301B2010E9438
:10790000945081110DC02FEF3FEF4FE75FE7C301A8
:10791000B2010E94034E18161CF48AE397E00CC0D3
:107920002FEF3FEF4FE75FE4C701B6010E94905091
:1079300018167CF48EE397E0FF90EF90DF90CF90E5
:10794000BF90AF909F908F907F906F905F904F907F
:107950002ACF2FEF3FEF4FE75FECC701B6010E9440
:10796000034E87FDE7CF20E030E0A901C701B60153
:107970000E94034E87FF08C08DE268DF4C01F7FAD2
:10798000F094F7F8F09402C0812C912CA12C60E0C7
:1079900070E080E09FE3AB1441F020E030E040E293
:1079A00051E40E94F74FA394F6CF9B01AC01C701AD
:1079B000B6010E94934F2B013C010E9464506B0161
:1079C0007C010E94074E9B01AC01C301B2010E94E1
:1079D000924F2B013C014AE0C701B601F7DE7C0162
:1079E000E80CF91CBB2021F08EE230DFE80EF91E16
:1079F000DB2CDD2019F120E030E040E251E4C3014E
:107A0000B2010E94684E2B013C010E9464504B0160
:107A1000A12CB12C4AE0C501B401D8DEE80EF91E54
:107A2000C501B4010E94074E9B01AC01C301B20124
:107A30000E94924F2B013C01DA94DBCFC701FF90EB
:107A4000EF90DF90CF90BF90AF909F908F907F90FE
:107A50006F905F904F900895789484B5826084BD54
:107A600084B5816084BD85B5826085BD85B5816042
:107A700085BD80916E00816080936E0010928100C0
:107A8000809181008260809381008091810081607B
:107A9000809381008091800081608093800080913C
:107AA000B10084608093B1008091B00081608093C8
:107AB000B00080919100826080939100809191004C
:107AC000816080939100809190008160809390000C
:107AD0008091A10082608093A1008091A1008160CB
:107AE0008093A1008091A00081608093A00080918C
:107AF0002101826080932101809121018160809326
:107B000021018091200181608093200180917A0081
:107B1000846080937A0080917A00826080937A00FA
:107B200080917A00816080937A0080917A008068E9
:107B300080937A001092C10061E086E30E949F0F5B
:107B400061E087E30E949F0F61E086E20E949F0F41
:107B500061E08AE10E949F0F61E08CE10E949F0F2B
:107B600061E088E10E949F0F62E083E00E949F0F26
:107B700062E082E00E949F0F62E080E10E949F0F1E
:107B800062E081E10E949F0F62E08FE10E949F0FFF
:107B900062E081E20E949F0F61E08CE30E949F0FF0
:107BA00061E08DE30E949F0F61E088E30E949F0FD8
:107BB00062E08EE00E949F0F62E08FE00E949F0FC4
:107BC00062E087E10E949F0F62E089E10E949F0FBF
:107BD00062E083E20E949F0F62E085E20E949F0FB5
:107BE00061E08EE20E949F0F61E080E30E949F0FA0
:107BF00061E08EE30E949F0F62E082E10E949F0F8E
:107C000062E083E10E949F0F62E08BE10E949F0F80
:107C100062E08DE10E949F0F62E087E20E949F0F69
:107C200062E089E20E949F0F61E08AE00E949F0F5C
:107C300061E088E00E949F0F61E089E00E949F0F51
:107C400061E08DE00E949F0F62E08FE30E949F0F32
:107C500062E08BE30E949F0F62E088E20E949F0F28
:107C600062E080E40E949F0F62E08AE20E949F0F20
:107C700062E08CE20E949F0F62E081E40E949F0F0D
:107C800062E082E40E949F0F62E084E30E949F0F03
:107C900062E085E30E949F0F62E080E00E949F0FF8
:107CA00062E081E00E949F0F62E089E30E949F0FE3
:107CB00062E08AE30E949F0F62E081E30E949F0FCF
:107CC00062E082E30E949F0F62E083E30E949F0FC5
:107CD00062E08BE20E949F0F62E08DE20E949F0FA4
:107CE00062E08FE20E949F0F62E080E20E949F0F9D
:107CF00061E084E00E949F0F61E085E00E949F0F99
:107D000061E086E00E949F0F61E08BE00E949F0F80
:107D100061E086E20E94AB0E61E088E10E94AB0E5A
:107D200061E088E30E94AB0E61E08EE30E94AB0E3F
:107D3000E091B80BF091B90B82E08083E091B40B35
:107D4000F091B50B1082E091B60BF091B70BD0E13A
:107D5000D0831092C00BE091BC0BF091BD0B86E07C
:107D60008083E091BA0BF091BB0B808180618083AE
:107D7000E091BA0BF091BB0B808188608083E09129
:107D8000BA0BF091BB0B808180688083E091BA0BC5
:107D9000F091BB0B80818F7D808364E670E080E092
:107DA00090E00E94E60F0E942E170E94C5130E94C9
:107DB000A7250E94681B0E941E1060937E0B709383
:107DC0007F0B8093800B9093810B87E091E39093DE
:107DD000430780934207C1E0C0936F00D0938100B6
:107DE00010928000C093DC0A80E092E09093DB0A5E
:107DF0008093DA0A909387008093860081E18093D4
:107E00008100109281001092850010928400809170
:107E1000DC0A8061809381000E941E1060937A0BBF
:107E200070937B0B80937C0B90937D0B0E941E10B4
:107E30006093820B7093830B8093840B9093850BDC
:107E40000E941E1060937E0B70937F0B8093800BBB
:107E50009093810B0E94473280915E0790915F075B
:107E6000A0916007B09161070197A105B10581F468
:107E70000E9447328091A6079091A707A091A8077A
:107E8000B091A9070197A105B10511F40C944E47D3
:107E90000E94473280915E0790915F07A091600732
:107EA000B09161070197A105B10581F40E944732A5
:107EB0008091A2079091A307A091A407B091A50774
:107EC0000197A105B10511F40C946D470E9447324A
:107ED00080915E0790915F07A0916007B091610764
:107EE0000197A105B10581F40E94473280919E0758
:107EF00090919F07A091A007B091A1070197A105BC
:107F0000B10511F40C948D4780E893E05EDCEFE757
:107F10002E2EE2E03E2EF5E7AF2EF2E0BF2E0E94BD
:107F20001E106093820B7093830B8093840B90934D
:107F3000850B00917E0B10917F0B2091800B30916F
:107F4000810B601771078207930748F460937E0BDB
:107F500070937F0B8093800B9093810B2CC0DC017E
:107F6000CB01801B910BA20BB30B883E9340A10564
:107F7000B10508F108511C4F2F4F3F4F00937E0B66
:107F800010937F0B2093800B3093810B0E94A725C9
:107F9000EC010E943312CE010C960E943312CE01E6
:107FA00048960E943312CE0184960E943312CE016D
:107FB000C0960E94331288EA9BE00E948E0B892BA8
:107FC00009F4BDC50E941E1060937A0B70937B0B61
:107FD00080937C0B90937D0B88EA9BE00E946C0B56
:107FE0008093790B982F9F7D953479F02091770BB2
:107FF0003091780BF901EB5BF44F80832F5F3F4F9B
:108000003093780B2093770B06C00E94DA1821E09A
:10801000DC011C962C938091770B9091780B813327
:10802000910564F02AE02093790BFC01EB5BF44F9F
:10803000208301969093780B8093770B8091790B36
:108040002091770B3091780B8A3039F4C901019770
:10805000A2E1BBE0E5E4FBE004C022333105B4F764
:108060006EC5AF0145545B40481759071CF4419158
:108070004D93F7CFFC01EE5EF44F108222303105B4
:108080000CF459C581E193E0A0DB8EE496E09DDB22
:108090008FE993E09ADB82E19BE097DB8FE993E045
:1080A00094DB8CE993E091DB8AE390E00E945C48EA
:1080B000EC011A821B821C821D821E821F8218867E
:1080C00019861A861B861C861D861E861F86188AA0
:1080D000198A1A8A1B8A1C8A1D8A1E8A1F8A188E70
:1080E000198E1A8E1B8E1C8E1D8E1E8E1F8E18A230
:1080F00019A21AA21BA21CA21DA21EA21FA218A690
:1081000019A61AA61BA61CA61DA61EA61FA618AA5F
:1081100019AA1AAA1BAA1CAA1DAA1EAA1FAA18AE2F
:1081200019AE68E072E082E19BE00E948C498C010C
:10813000FC0180818654823008F027C161EA73E037
:10814000C8010E94B051892B09F4D3C064EA73E0DE
:10815000C8010E94B051892B09F4CBC068EA73E0D2
:10816000C8010E94B051892B09F4C6C06BEA73E0C4
:10817000C8010E94B051892B09F4BEC06FEA73E0B8
:10818000C8010E94B051892B09F4B9C063EB73E0B8
:10819000C8010E94B051892B09F4B4C067EB73E0A9
:1081A000C8010E94B051892B09F4ACC06AEB73E09E
:1081B000C8010E94B051892B09F4A7C06EEB73E08F
:1081C000C8010E94B051892B09F4A2C062EC73E08F
:1081D000C8010E94B051892B09F49DC066EC73E080
:1081E000C8010E94B051892B09F498C06AEC73E071
:1081F000C8010E94B051892B09F493C06EEC73E062
:10820000C8010E94B051892B09F48EC062ED73E061
:10821000C8010E94B051892B09F489C066ED73E052
:10822000C8010E94B051892B09F484C06AED73E043
:10823000C8010E94B051892B09F47FC06EED73E034
:10824000C8010E94B051892B09F47AC062EE73E034
:10825000C8010E94B051892B09F475C066EE73E025
:10826000C8010E94B051892B09F470C06AEE73E016
:10827000C8010E94B051892B09F46BC06EEE73E007
:10828000C8010E94B051892B09F466C062EF73E007
:10829000C8010E94B051892B09F461C066EF73E0F8
:1082A000C8010E94B051892B09F45CC06AEF73E0E9
:1082B000C8010E94B051892B09F457C06EEF73E0DA
:1082C000C8010E94B051892B09F452C062E074E0E9
:1082D000C8010E94B051892B09F44DC066E074E0DA
:1082E000C8010E94B051892B09F448C08FEF9FEF5D
:1082F00047C080E090E044C081E090E041C08CE164
:1083000090E03EC08DE690E03BC08FE690E038C044
:1083100080E790E035C081E790E032C082E790E0EE
:108320002FC083E790E02CC084E790E029C088E765
:1083300090E026C089E790E023C08AE790E020C063
:1083400083E890E01DC084E890E01AC08DE890E0DA
:1083500017C08EE890E014C08FE890E011C080E96B
:1083600090E00EC081EA90E00BC085EB90E008C081
:1083700086EB90E005C087EB90E002C088EB90E0D0
:108380009093010280930002BBC08FEF9FEF909308
:10839000010280930002B8C0D8018C91883539F46D
:1083A000C8010196B6D76A837B838C839D83F801CD
:1083B0008081893539F4C8010196ABD76E837F83FC
:1083C00088879987D8018C918A3539F4C80101963C
:1083D000A0D76A877B878C879D87F801808181344D
:1083E00049F4C801019695D70E945F506E877F8738
:1083F000888B998BD8018C91823449F4C8010196FD
:1084000088D70E945F506A8B7B8B8C8B9D8BF80189
:108410008081833449F4C80101967BD70E945F5064
:108420006E8B7F8B888F998FD8018C91833539F42F
:10843000C80101966ED76A8F7B8F8C8F9D8FF80154
:108440008081803549F4C801019663D70E945F504E
:108450006E8F7F8F88A399A3D8018C91863549F4BC
:10846000C801019656D70E945F506AA37BA38CA3D4
:108470009DA3F8018081873549F4C801019649D749
:108480000E945F506EA37FA388A799A7D8018C9103
:10849000853449F4C80101963CD70E945F506AA711
:1084A0007BA78CA79DA7F8018081843549F4C8017A
:1084B00001962FD70E945F506EA77FA788AB99AB1C
:1084C000D8018C918D3449F4C801019622D70E94BD
:1084D0005F506AAB7BAB8CAB9DABF8018081813583
:1084E00049F4C801019615D70E945F506EAB7FAB6F
:1084F00088AF99AF6AE074E080E090E00DD78C011E
:108500000115110509F048CF0E94DA18DC011C960C
:108510001C910E94473240906A0750906B07609010
:108520006C0770906D07CEA8DFA8E8ACF9AC0E948C
:10853000DA18C0924607D0924707E0924807F092B7
:10854000490780910002909101029924939482300E
:10855000910538F09C012F5631092630310508F07D
:10856000912C112371F08D36910559F09C012857FB
:1085700031092330310528F0855B9109039708F014
:10858000D0C20E94473280915E0790915F07A09110
:108590006007B09161070197A105B10529F0992005
:1085A00019F08DEF92E0BFC2209719F489EF92E0A5
:1085B000BAC2E0900002F0900102BFEFEB16FB069A
:1085C000A9F3E114F104B9F48091DD0A9091DE0A77
:1085D000892B61F482E090E06FD521E132E0FC016B
:1085E000318320839093DE0A8093DD0A0091DD0AB7
:1085F0001091DE0A6EC0FCE1EF16F104B9F480912F
:10860000DF0A9091E00A892B61F482E090E054D572
:108610002BE132E0DC012D933C939093E00A8093B0
:10862000DF0A0091DF0A1091E00A53C0BDE6EB16A5
:10863000F104B9F48091E10A9091E20A892B61F486
:1086400082E090E039D525E232E0FC0131832083DD
:108650009093E20A8093E10A0091E10A1091E20A04
:1086600053C0FFE6EF16F104B9F48091E30A90914C
:10867000E40A892B61F482E090E01ED52FE232E01B
:10868000DC012D933C939093E40A8093E30A0091DC
:10869000E30A1091E40A53C000E010E0B0E7EB16E3
:1086A000F104B9F48091E50A9091E60A892B61F40E
:1086B00082E090E001D529E332E0FC0131832083A0
:1086C0009093E60A8093E50A0091E50A1091E60A84
:1086D0006CC0F1E7EF16F104B9F48091E70A9091CC
:1086E000E80A892B61F482E090E0E6D423E432E0EA
:1086F000DC012D933C939093E80A8093E70A009164
:10870000E70A1091E80A6CC0B2E7EB16F104B9F47D
:108710008091E90A9091EA0A892B61F482E090E065
:10872000CBD42DE432E0FC01318320839093EA0A1C
:108730008093E90A0091E90A1091EA0A6AC0F3E716
:10874000EF16F104B9F48091EB0A9091EC0A892BB1
:1087500061F482E090E0B0D427E532E0DC012D93B3
:108760003C939093EC0A8093EB0A0091EB0A1091F2
:10877000EC0A68C0B4E7EB16F104B9F48091ED0A95
:108780009091EE0A892B61F482E090E095D421E685
:1087900032E0FC01318320839093EE0A8093ED0A4E
:1087A0000091ED0A1091EE0A68C0F8E7EF16F104A7
:1087B000B9F48091EF0A9091F00A892B61F482E07C
:1087C00090E07AD42BE632E0DC012D933C93909339
:1087D000F00A8093EF0A0091EF0A1091F00A68C046
:1087E000B9E7EB16F104A9F48091F10A9091F20A2D
:1087F000892B51F482E090E05FD4FC01B182A08229
:108800009093F20A8093F10A0091F10A1091F20A12
:108810006AC0FAE7EF16F104A9F48091F30A909187
:10882000F40A892B51F482E090E046D4DC012D92C9
:108830003C929093F40A8093F30A0091F30A10910A
:10884000F40A6CC0BDE8EB16F104B9F48091F50AA6
:108850009091F60A892B61F482E090E02DD429E80A
:1088600032E0FC01318320839093F60A8093F50A6D
:108870000091F50A1091F60A6CC03EE8E316F10487
:10888000B9F48091F70A9091F80A892B61F482E09B
:1088900090E012D4E3E9F2E0DC01ED93FC939093D5
:1088A000F80A8093F70A0091F70A1091F80A6CC051
:1088B000FFE8EF16F104B9F48091F90A9091FA0AF1
:1088C000892B61F482E090E0F7D3EDE9F2E0DC017E
:1088D000ED93FC939093FA0A8093F90A0091F90AB8
:1088E0001091FA0A6CC0F0E9EF16F104B9F4809126
:1088F000FB0A9091FC0A892B61F482E090E0DCD3C2
:10890000E7EAF2E0DC01ED93FC939093FC0A80939C
:10891000FB0A0091FB0A1091FC0A6CC0F1EAEF1609
:10892000F104B9F48091FD0A9091FE0A892B61F45B
:1089300082E090E0C1D3E1EBF2E0DC01ED93FC9347
:108940009093FE0A8093FD0A0091FD0A1091FE0AA1
:108950006BC0F5EBEF16F104B9F48091FF0A90912A
:10896000000B892B61F482E090E0A6D3EBEBF2E000
:10897000DC01ED93FC939093000B8093FF0A009130
:10898000FF0A1091000B50C0F6EBEF16F104B9F49A
:108990008091010B9091020B892B61F482E090E0B1
:1089A0008BD3E5ECF2E0DC01ED93FC939093020BAA
:1089B0008093010B0091010B1091020B35C0F7EB76
:1089C000EF16F104B9F48091030B9091040B892BFD
:1089D00061F482E090E070D3EFECF2E0DC01ED9323
:1089E000FC939093040B8093030B0091030B109165
:1089F000040B1AC0F8EBEF16F104B1F48091050BEB
:108A00009091060B892B61F482E090E055D3E3EE60
:108A1000F2E0DC01ED93FC939093060B8093050B41
:108A20000091050B1091060B0115110589F489EFD2
:108A300092E00E94E53B0E94DA180E94E4178EE063
:108A400094E00E94D33B8CE993E00E94D33B71C039
:108A500085EF92E00E94E53B0E94DA180E94E4173D
:108A60000E94DA181092450710924407E12CF12C6D
:108A7000FFEFEF1AFF0A21E0E216F10441F081EF67
:108A800092E00E94E53B0E94DA180E94E417D801A8
:108A9000ED91FC910480F581E02DBE01C80119958E
:108AA0000E94DA18C0904407D09045070E94DA1857
:108AB000FC018485E114F104D9F281110AC0E414A7
:108AC000F5043CF4C114D10421F0F2E0CF16D10436
:108AD00079F688EA9BE00E948E0B181619062CF492
:108AE00088EA9BE00E946C0BF4CFCD2809F438C2D1
:108AF000992009F432C20E94473280916607909112
:108B00006707A0916807B09169070197A105B105B2
:108B100009F023C20E94DA1821E0DC011C962C9394
:108B20001CC281E093E00E94E53B0E94DA180E949B
:108B3000E417CE0156D31092780B1092770B8091E8
:108B4000110B8111AAC00E94DA18FC0184858823C8
:108B500009F4A3C00E942E17EC01FC01E253FD4F63
:108B6000108240960E947426CE0186579F4F0E9425
:108B70007426CE018C5F9E4F0E9474260E946F3532
:108B80007C018C01075C1F4FC1E0D0E06801F8E375
:108B9000CF1AD108D6018C918823D9F084E294E0D1
:108BA0000E94E53B88E294E00E94E53BCE010E94F2
:108BB000583C8CE993E00E94E53B60E08C2F0E94DA
:108BC000AB0E40E050E0BE01C7010E94D932F60171
:108BD0001082D8018C918823F9F084E294E00E94FD
:108BE000E53B8FE394E00E94E53BCE010E94583CB8
:108BF0008CE993E00E94E53B61E08C2F0E949F0F7F
:108C000060E08C2F0E94AB0E41E050E0BE01C70136
:108C10000E94D932F801108221960F5F1F4FC53391
:108C2000D10509F0B3CF0E94C6328091DE0C90E0EE
:108C30009C01220F331F820F931FFC01E35BF34F54
:108C400080818F7B80838091E10C90E09C01220FDA
:108C5000331F820F931FFC01E35BF34F80818F7BF7
:108C600080838091E40C90E09C01220F331F820FDF
:108C7000931FFC01E35BF34F80818F7B80838091A6
:108C8000E70C90E09C01220F331F820F931FFC0121
:108C9000E35BF34F80818F7B80830E94DA18DC01D5
:108CA0001C968C918093110BC0910F0BD091100BDF
:108CB0000E944732FC0182819381C817D90799F03D
:108CC0000E944732DC0112968D919C9113979093EC
:108CD000100B80930F0B0E942E170E94C5130E9449
:108CE000A7250E94681B0E941E1060930B0B7093B7
:108CF0000C0B80930D0B90930E0B00917A0B10913F
:108D00007B0B20917C0B30917D0B601771078207E4
:108D1000930708F4B6C0DC01CB01801B910BA20BBA
:108D2000B30B89389341A105B10508F4B4C00E9482
:108D3000DA18DC011C968C91882319F08DE093E001
:108D400002C089E093E00E94E53B0E94DA180E948D
:108D5000E4170E942E17EC01FC01E755FD4F8081BE
:108D6000882341F0CE0182589E4F0E9479366B01D4
:108D70007C0107C0FE01E25BFF4FC080D180E28032
:108D8000F3800E94DA18C0924A07D0924B07E09213
:108D90004C07F0924D07FE01E655FD4F8081882378
:108DA00041F0CE0184569E4F0E9479366B017C01C2
:108DB00007C0FE01E853FF4FC080D180E280F380FE
:108DC0000E94DA18C0924E07D0924F07E0925007E7
:108DD000F0925107FE01E555FD4F8081882341F057
:108DE000CE0186549E4F0E9479366B017C0106C0ED
:108DF000CE5BDE4FC880D980EA80FB800E94DA1803
:108E0000C0925207D0925307E0925407F092550750
:108E10000E94DA180E9437180E942E170E94C1196A
:108E20000E94DA180E94211B0E94DA180E94F6178D
:108E30000E94473280915E0790915F07A091600782
:108E4000B09161070197A105B10541F085E093E07C
:108E50000E94E53B0E94DA180E94E4178091070BFC
:108E60009091080BA091090BB0910A0B0196A11DDE
:108E7000B11D8093070B9093080BA093090BB0933F
:108E80000A0B0E941E1060937A0B70937B0B8093E9
:108E90007C0B90937D0B0E942B0C41C885E594E0E0
:108EA0000E94E53B0E942E17CF931F921F921F92A4
:108EB0001F92812C912CA12CB12CC12CD12C76018C
:108EC00097018601B701A6010E94D5020F900F906D
:108ED0000F900F900F900C94483F8DE694E00E9405
:108EE000E53B0E942E171F9221E02F931F921F92A5
:108EF0001F92812C912CA12CB12CC12CD12C76014C
:108F000097018601B701A6010E94D5020F900F902C
:108F10000F900F900F900C94663F85E894E00E94AC
:108F2000E53B0E942E171F921F9221E02F931F9264
:108F30001F92812C912CA12CB12CC12CD12C76010B
:108F400097018601B701A6010E94D5020F900F90EC
:108F50000F900F900F900C94843F89EE92E002C026
:108F60008DEE92E00E94E53B0E94DA180E94E41721
:108F70000E94DA181092460710924707109248078D
:108F800010924907D6CD8091450C9091460C29C18D
:108F90001092AB0B1092AA0B88EE93E0A0E0B0E029
:108FA0008093AC0B9093AD0BA093AE0BB093AF0B33
:108FB0008AE693E09093A90B8093A80B85EC90E050
:108FC0009093B50B8093B40B84EC90E09093B70B27
:108FD0008093B60B80EC90E09093B90B8093B80B24
:108FE00081EC90E09093BB0B8093BA0B82EC90E005
:108FF0009093BD0B8093BC0B86EC90E09093BF0BDD
:109000008093BE0B1092C10B1092C20B1092C30B37
:109010001092C40B82E090E04FD02CE733E0FC01CB
:109020003183208390934C0C80934B0C6EE973E05A
:1090300085E49CE00E94100E8091DD0CAEEDBCE05A
:109040009FEF48EB5BE0803378F48C93282F30E07F
:10905000F901EE0FFF1F2E0F3F1FF901E35BF34FE6
:10906000528341838F5F01C09C931396FCE0AA3E1C
:10907000BF0749F78093DD0C0895EF920F931F937C
:10908000CF93DF93E80147FD02C034E001C034E133
:10909000E42F440FFF0BF7FF03C0F195E195F109B1
:1090A000E32E022F2E2FAE01B3D1CE01DF91CF914F
:1090B0001F910F91EF900895CF93DF938230910528
:1090C00010F482E090E0E091EE0CF091EF0C20E0E3
:1090D00030E0C0E0D0E0309711F140815181481775
:1090E0005907C0F04817590761F48281938120978E
:1090F00019F09B838A832BC09093EF0C8093EE0C26
:1091000026C02115310519F04217530718F49A01AA
:10911000BE01DF01EF010280F381E02DDCCF2115DC
:10912000310509F1281B390B2430310590F41296D2
:109130008D919C9113976115710521F0FB0193832B
:10914000828304C09093EF0C8093EE0CFD01329665
:1091500044C0FD01E20FF31F819391932250310926
:109160002D933C933AC02091EC0C3091ED0C232BC5
:1091700041F420910402309105023093ED0C2093CC
:10918000EC0C20910202309103022115310541F4CB
:109190002DB73EB74091060250910702241B350BB4
:1091A000E091EC0CF091ED0CE217F307A0F42E1B0C
:1091B0003F0B2817390778F0AC014E5F5F4F24173B
:1091C000350748F04E0F5F1F5093ED0C4093EC0CA9
:1091D0008193919302C0E0E0F0E0CF01DF91CF9165
:1091E00008950F931F93CF93DF93009709F48CC0DA
:1091F000FC013297138212820091EE0C1091EF0C59
:109200000115110581F420813181820F931F209176
:10921000EC0C3091ED0C2817390779F5F093ED0C33
:10922000E093EC0C71C0D80140E050E0AE17BF07EE
:1092300050F412962D913C911397AD0121153105F3
:1092400009F1D901F3CF9D01DA01338322836081D3
:109250007181860F971F8217930769F4EC012881AB
:109260003981260F371F2E5F3F4F318320838A813C
:109270009B8193838283452B29F4F093EF0CE09339
:10928000EE0C42C01396FC93EE931297ED014991B8
:1092900059919E01240F351FE217F30771F4808165
:1092A0009181840F951F029611969C938E938281D3
:1092B000938113969C938E931297E0E0F0E0D8018F
:1092C00012968D919C911397009719F0F8018C01DB
:1092D000F6CF8D919C9198012E5F3F4F820F931F87
:1092E0002091EC0C3091ED0C2817390769F4309778
:1092F00029F41092EF0C1092EE0C02C0138212822D
:109300001093ED0C0093EC0CDF91CF911F910F9116
:1093100008956627772709C24AEE5CE000C0FA018B
:10932000A191B081009719F41097E1F0CD01DC0113
:10933000CD010D90002011F4C00113C0FB0121915B
:10934000222319F02015D9F7F3CFFB012191201525
:1093500019F41E92119606C02223C1F70D90002029
:10936000A1F7D001FA01A193B0830895BB274A3039
:1093700031F4992322F4BDE2909581959F4F30C03E
:10938000BB272A3051F4992342F4BDE29095809591
:10939000709561957F4F8F4F9F4F01C0BB27FA019A
:1093A000A62F6217710581059105330B30FB66F01E
:1093B000AA27660F771F881F991FAA1FA21710F0F0
:1093C000A21B63953850A9F7A05DAA3308F0A95DE8
:1093D000A19336F7B111B1931082CA0104C4BB271F
:1093E000FB015527AA27880F991FAA1FA41710F061
:1093F000A41B83955051B9F7A05DAA3308F0A95D6D
:10940000A193009779F7B111B1931192CB01EBC3FE
:109410004F925F926F927F929F92AF92BF92CF9244
:10942000DF92EF92FF920F931F93CF93DF93CDB70D
:10943000DEB729970FB6F894DEBF0FBECDBF6A0125
:10944000122FB02E2BE3201720F0FF24F394F00E00
:1094500002C0BCE3FB2E0F2D27E0AE014F5F5F4F34
:10946000CAD2AC018981982F9970913031F0E1FC1A
:1094700006C0E0FE06C090E205C09DE203C09BE28C
:1094800001C090E0EE2DE07183FF3CC0911102C05D
:1094900083E001C084E0811718F4212F281B01C04C
:1094A00020E0E1110BC0F601822F30E2882319F091
:1094B00031938150FBCFC20ED11C20E0992329F0BB
:1094C000D6019C93F60131966F01C6010396E2FE28
:1094D0000AC03EE4D6013C9341E411964C931197A7
:1094E00012963C9306C03EE6F601308341E6418386
:1094F0003283FC01322F40E2332309F442C041930E
:109500003150FACF82FF44C0911102C083E001C004
:1095100084E0811718F4212F281B01C020E0E111FD
:109520000BC0F601822F30E2882319F0319381506D
:10953000FBCFC20ED11C20E0992329F0D6019C93C9
:10954000F60131966F01C6010396E2FE0BC039E4C5
:10955000D6013C933EE411963C93119736E4129663
:109560003C9307C039E6F60130833EE6318336E6A8
:109570003283FC01322F40E2332319F04193315002
:10958000FBCFFC01E20FF11D10828EEF9FEFB7C001
:10959000F1E0911101C0F0E06F2F70E01416150694
:1095A00024F49A012F5F3F4F02C021E030E0260FE4
:1095B000371FBB2029F06B2D70E06F5F7F4F02C01B
:1095C00060E070E0260F371F612F70E02617370725
:1095D0001CF4121B212F01C020E03E2D387159F4DC
:1095E000D601322F60E2332319F06D933150FBCF57
:1095F000C20ED11C20E0FF2331F0D6019C93B601AE
:109600006F5F7F4F6B01E1110BC0F601922F30E3CA
:10961000992319F031939150FBCFC20ED11C20E059
:109620009F2D940F3A81782F7071A72E84FF03C06D
:10963000313309F49150191624F4993018F098E058
:1096400001C091E0E42F852F57FF02C0E0E080E0E9
:109650006E2F782FE0E0F0E0AEE29A2E3A01691A20
:1096600071082A01461A570A0B2D10E01195019531
:1096700011096F3F8FEF780729F4D6019C92C6013C
:1096800001966C014617570784F0661677066CF44E
:109690007F01E40CF51CA1E0B0E0AC0FBD1FEA0EA9
:1096A000FB1ED7011196BC9002C090E3B92E615009
:1096B00071093196C60101967C016017710724F08B
:1096C000D601BC926C01D5CF6417750741F43633CF
:1096D00020F4353321F4A11002C081E3B82EF60145
:1096E000B082F701822F90E2882319F09193815084
:1096F000FBCFF701E20FF11D108280E090E0299688
:109700000FB6F894DEBF0FBECDBFDF91CF911F9192
:109710000F91FF90EF90DF90CF90BF90AF909F9010
:109720007F906F905F904F9008956F927F928F928D
:109730009F92AF92BF92CF92DF92EF92FF920F93E0
:109740001F93CF93DF93EC017B016115710519F035
:10975000DB018D939C938E010F5F1F4F7880872DC7
:1097600090E021D2892B11F0E801F5CFBDE27B1208
:1097700005C00F5F1F4F7980C1E008C0EBE27E1289
:1097800004C08E010E5F1F4F7980C0E06801F1E0D8
:10979000CF1AD10843E050E064EF72E0C6010BD26B
:1097A000892BE9F4680122E0C20ED11C45E050E0AB
:1097B0006FEE72E0C601FFD1892B21F4680187E0CA
:1097C000C80ED11CE114F10419F0D701CD92DC923E
:1097D000C111F9C060E070E080E89FE7FDC043E0A0
:1097E00050E06CEE72E0C601E6D1892B51F4E11431
:1097F000F10409F4EDC00E5F1F4FF70111830083E0
:10980000E7C0680160E070E0CB0100E010E0F60125
:10981000D0EDD70DDA3050F52C2F2260622E2C2F90
:109820002870C2FF05C0211127C00F5F1F4F24C041
:10983000222311F001501109A5E0B0E09B01AC0119
:1098400030D34B015C01880C991CAA1CBB1CC501C0
:10985000B4016D0F711D811D911D6839A9E97A0749
:109860008A07A9E19A0740F0C66005C0DE3F51F4BF
:10987000C3FD44C0C8606C2EBFEFCB1ADB0A7080FA
:10988000C62DC5CF2D2F2F7D2531C1F540814D32FD
:1098900011F4C06106C04B3221F0319621E030E076
:1098A00006C03296D60111964C9122E030E0A0ED30
:1098B000A40FAA3018F0E21BF30B20C040E050E0E8
:1098C0004038BCE05B075CF49A01220F331F220F83
:1098D000331F420F531F440F551F4A0F511D31961E
:1098E000DF0111972C91A0EDA20FAA3048F3C4FF1D
:1098F00003C0519541955109040F151FC1FF07C0C1
:10990000E114F10421F03197D701ED93FC937FD15D
:10991000C370C33019F06B017C0106C06B017C0180
:10992000F7FAF094F7F8F09420E030E0A901C701CD
:10993000B60169D1882309F443C017FF06C0119509
:1099400001951109CBE0D3E002C0C3E2D3E05E0190
:10995000B8E1AB1AB1084601BE2DAF2D90E2E92E59
:10996000F12C0E151F057CF0FE01259135914591D6
:109970005491B4018B2F9A2FABD14B01B82FA92F43
:109980000E191F09EECF2497F594E794CA15DB054D
:1099900041F76401EB2EFA2E8E2D880F8F2D881F34
:1099A0008F3F41F020E030E0A901C701B6012BD183
:1099B000811106C082E290E09093F10C8093F00C4C
:1099C000C701B60109C060E070E080E89FEF04C005
:1099D00060E070E080EC9FE7DF91CF911F910F91E5
:1099E000FF90EF90DF90CF90BF90AF909F908F90BF
:1099F0007F906F900895283008F027E03327DA0130
:109A0000990F311D87FD916000966105710539F44C
:109A100032602E5F3D9330E32A95E1F708959F3F32
:109A200030F080387105610509F03C5F3C5F3D9383
:109A3000913008F08068911DDF93CF931F930F93AF
:109A4000FF92EF92192F987F9695E92F969596950C
:109A5000E90FFF27EF57FC4F99273327EE24FF2408
:109A6000A701E70105900894079428F4360FE71E34
:109A7000F81E491F511D660F771F881F991F0694F6
:109A8000A1F70590079428F4E70EF81E491F561F0A
:109A9000C11D770F881F991F661F0694A1F70590B7
:109AA000079428F4F80E491F561FC71FD11D880FB1
:109AB000991F661F771F0694A1F70590079420F45D
:109AC000490F561FC71FD81F990F661F771F881F82
:109AD0000694A9F784911095177041F0D695C79513
:109AE00057954795F794E7941A95C1F7E7E2F3E0A5
:109AF00068941590159135916591959105907FE247
:109B00007395E118F10A430B560BC90BD009C0F746
:109B1000E10CF11E431F561FC91FD01D7EF4703388
:109B200011F48A95E6CFE894015030F0080F0AF45A
:109B30000027021708F4202F2395022F7A3328F0EC
:109B400079E37D932A95E9F710C07D932A9589F6EC
:109B5000069497956795379517951794E118F10A2C
:109B6000430B560BC90BD00998F023957E91739542
:109B70007A3308F070E37C932013B8F77E9170611C
:109B80007D9330F0839571E37D9370E32A95E1F73F
:109B90001124EF90FF900F911F91CF91DF919927A2
:109BA00087FD909508959111F6C0803219F0895083
:109BB0008550D0F70895FB01DC014150504088F0FA
:109BC0008D9181341CF08B350CF4805E659161348D
:109BD0001CF06B350CF4605E861B611171F3990B00
:109BE0000895881BFCCFDC01FC01672F719177235E
:109BF000E1F7329704C07C916D9370836291AE1748
:109C0000BF07C8F3089540D008F481E00895E894B0
:109C100009C097FB3EF490958095709561957F4FB4
:109C20008F4F9F4F9923A9F0F92F96E9BB27939562
:109C3000F695879577956795B795F111F8CFFAF472
:109C4000BB0F11F460FF1BC06F5F7F4F8F4F9F4FA3
:109C500016C0882311F096E911C0772321F09EE801
:109C6000872F762F05C0662371F096E8862F70E067
:109C700060E02AF09A95660F771F881FDAF7880F41
:109C80009695879597F90895990F0008550FAA0B97
:109C9000E0E8FEEF16161706E807F907C0F01216FF
:109CA0001306E407F50798F0621B730B840B950B02
:109CB00039F40A2661F0232B242B252B21F4089557
:109CC0000A2609F4A140A6958FEF811D811D0895F4
:109CD0000BD07BC06CD028F071D018F0952309F020
:109CE0005DC062C01124A5C081D0A0F3959FD1F3BF
:109CF000950F50E0551F629FF001729FBB27F00D3A
:109D0000B11D639FAA27F00DB11DAA1F649F66278E
:109D1000B00DA11D661F829F2227B00DA11D621FDD
:109D2000739FB00DA11D621F839FA00D611D221F97
:109D3000749F3327A00D611D231F849F600D211D7B
:109D4000822F762F6A2F11249F5750408AF0E1F01E
:109D500088234AF0EE0FFF1FBB1F661F771F881F67
:109D600091505040A9F79E3F510570F017C061C057
:109D70005F3FECF3983EDCF3869577956795B79552
:109D8000F795E7959F5FC1F7FE2B880F911D96957C
:109D9000879597F9089599278827089597F99F67D8
:109DA00080E870E060E008959FEF80EC0895002463
:109DB0000A941616170618060906089500240A9430
:109DC00012161306140605060895092E0394000CB6
:109DD00011F4882352F0BB0F40F4BF2B11F460FF45
:109DE00004C06F5F7F4F8F4F9F4F089557FD90586E
:109DF000440F551F59F05F3F71F04795880F97FB4F
:109E0000991F61F09F3F79F0879508951216130608
:109E10001406551FF2CF4695F1DF08C01616170637
:109E20001806991FF1CF869571056105089408956C
:109E3000E894BB2766277727CB0197F90895F9990E
:109E4000FECF92BD81BDF89A992780B50895262F3F
:109E5000F999FECF1FBA92BD81BD20BD0FB6F8940F
:109E6000FA9AF99A0FBE01960895052E97FB16F4FB
:109E700000940FD057FD05D024D007FC02D046F443
:109E800008C050954095309521953F4F4F4F5F4FFB
:109E9000089590958095709561957F4F8F4F9F4F56
:109EA000089531D0A59F900DB49F900DA49F800D73
:109EB000911D11240895B7FFF4CFF3DF821B930B9C
:109EC0000895A1E21A2EAA1BBB1BFD010DC0AA1FFB
:109ED000BB1FEE1FFF1FA217B307E407F50720F013
:109EE000A21BB30BE40BF50B661F771F881F991F8E
:109EF0001A9469F760957095809590959B01AC01D7
:109F0000BD01CF010895A29FB001B39FC001A39FDF
:109F1000700D811D1124911DB29F700D811D1124A2
:109F2000911D08955058BB27AA270ED04ECF3FDF72
:109F300030F044DF20F031F49F3F11F41EF434CFB1
:109F40000EF4E095E7FB2ACFE92F50DF80F3BA1734
:109F5000620773078407950718F071F49EF568CFC0
:109F60000EF4E0950B2EBA2FA02D0B01B901900134
:109F70000C01CA01A0011124FF27591B99F0593F78
:109F800050F4503E68F11A16F040A22F232F342FC0
:109F90004427585FF3CF469537952795A795F0400E
:109FA0005395C9F77EF41F16BA0B620B730B840B23
:109FB000BAF09150A1F0FF0FBB1F661F771F881FDB
:109FC000C2F70EC0BA0F621F731F841F48F4879533
:109FD00077956795B795F7959E3F08F0B3CF939522
:109FE000880F08F09927EE0F9795879508950CD064
:109FF000ECCEE4DE40F0DBDE30F021F45F3F19F020
:10A00000CDCE511116CFD0CEF1DE98F39923C9F3FE
:10A010005523B1F3951B550BBB27AA27621773076E
:10A02000840738F09F5F5F4F220F331F441FAA1F22
:10A03000A9F333D00E2E3AF0E0E830D091505040E2
:10A04000E695001CCAF729D0FE2F27D0660F771F90
:10A05000881FBB1F261737074807AB07B0E809F072
:10A06000BB0B802DBF01FF2793585F4F2AF09E3F07
:10A07000510568F093CEDDCE5F3FECF3983EDCF304
:10A08000869577956795B795F7959F5FC9F7880F80
:10A09000911D9695879597F90895E1E0660F771FD2
:10A0A000881FBB1F621773078407BA0720F0621B63
:10A0B000730B840BBA0BEE1F88F7E095089504D05C
:10A0C0006894B111B6CE089599DE88F09F5790F04C
:10A0D000B92F9927B751A0F0D1F0660F771F881FCD
:10A0E000991F1AF0BA95C9F712C0B13081F0A0DEFD
:10A0F000B1E008959DCE672F782F8827B85F39F09B
:10A10000B93FCCF3869577956795B395D9F73EF42B
:10A1100090958095709561957F4F8F4F9F4F0895D3
:10A12000B3DD08F48FEF0895AFDD880B990B089528
:10A13000DB018F939F93B5DEBF91AF91A29F800DFE
:10A14000911DA39F900DB29F900D11240895991B0E
:10A1500079E004C0991F961708F0961B881F7A951E
:10A16000C9F780950895EE0FFF1F881F8BBF0790DA
:10A17000F691E02D19946F927F928F929F92AF92F9
:10A18000BF92CF92DF92EF92FF920F931F93CF93E4
:10A19000DF93EC01009789F4CB01DF91CF911F9100
:10A1A0000F91FF90EF90DF90CF90BF90AF909F9076
:10A1B0008F907F906F900C945C48FC01E60FF71F26
:10A1C0009C0122503109E217F30708F4ABC0D90112
:10A1D0000D911C91119706171707B0F00530110566
:10A1E00008F49EC0C80104978617970708F498C022
:10A1F00002501109061B170B019311936D937C9369
:10A20000CF010E94F1488CC05B01A01AB10A4C0139
:10A21000800E911EA091EE0CB091EF0C40E050E04A
:10A22000E12CF12C109709F44AC0A815B905D1F515
:10A230006D907C901197630182E0C80ED11CCA1406
:10A24000DB0480F1A3014A195B096A0182E0C80EB0
:10A25000D11C1296BC9012971396AC91B5E0CB1618
:10A26000D10440F0B282A38351834083D9016D931E
:10A270007C930AC00E5F1F4FC301800F911FF9012D
:10A2800091838083EB2DFA2FE114F10431F0D70193
:10A290001396FC93EE93129743C0F093EF0CE09368
:10A2A000EE0C3EC08D919C9111974817590708F408
:10A2B000AC017D0112960D90BC91A02DB3CF809181
:10A2C000EC0C9091ED0C88159905E1F446175707B1
:10A2D000C8F48091020290910302009741F48DB777
:10A2E0009EB74091060250910702841B950BE81718
:10A2F000F907C0F4F093ED0CE093EC0CF9017183D5
:10A3000060830EC0CB010E945C487C01009751F035
:10A31000A801BE011CD0CE010E94F148C70104C0B3
:10A32000CE0102C080E090E0DF91CF911F910F91AC
:10A33000FF90EF90DF90CF90BF90AF909F908F9065
:10A340007F906F90089581E090E0F89419C0FB0130
:10A35000DC0102C001900D9241505040D8F70895A1
:10A36000FB01DC018D91019080190110D9F3990B4B
:10A370000895FB01DC0101900D920020E1F70895A2
:10A3800012E0C2EAD2E000E005C0802FFE01EBDE61
:10A390002196011DC33AD10780E00807B1F7F89470
:02A3A000FFCFED
:10A3A200FFFF0000F20C8000200A0D0000000000F8
:10A3B200009C17C1134717000000009D17C31376B6
:10A3C2001A00000000C5366634683500000000D669
:10A3D2002500254C2500000000CA12E20C440D00A5
:10A3E200000000C5329C3085310000000010365854
:10A3F200346A3400000000C4366434A23400000021
:10A40200003212E00C0B0D00000000C1365E343841
:10A412003500000000712B04259825000000001172
:10A42200365A34DA3400000000C6366834F3350098
:10A4320000000012365C34C93500000000C33662E9
:10A4420034DD35000000000F3656348E3500000032
:10A4520000D425FC24062500000000C332983045B4
:10A462003300000000D72502257D2500000000C230
:10A472003660345B3500000000D525FE24E124005F
:10A48200000000C4329A309E3052303300523032D3
:10A4920000523037005230310052303900523838D1
:10A4A20000523837005238380052303000523837B4
:10A4B20000523038005231330052313200523131C1
:10A4C200005237330052373200523731005231379F
:10A4D2000052313600523135000100000001000007
:10A4E2000001000000523835005238340052303535
:10A4F2000052303600362E342E322E5200005230A8
:10A5020034005238370000000000C40B2E0B5D0BE4
:10A512000A0C8E0B6C0B800B000000000E365434BC
:10A522005239392041524455494E4F2053544152D9
:10A5320054555020434F4D504C4554450D0A002A66
:10A542000047300047303000473100473031004784
:10A552003238004630390046390046313100463142
:10A56200320046313300463134004631350046313F
:10A57200360046323000463231004632320046332F
:10A58200310046333200463431004634320046341C
:10A5920033004634340046363100463831004638FE
:10A5A20032004638330046383400200A0D00523952
:10A5B200392068616E646C6572203D3D204E554CB9
:10A5C2004C0D0A0052393900207265736574746942
:10A5D2006E67206469676974616C2070696E00201F
:10A5E200726573657474696E6720616E616C6F6702
:10A5F2002070696E0052393920484F4D45205A204B
:10A602004F4E20535441525455500D0A005239397D
:10A6120020484F4D452059204F4E2053544152540B
:10A6220055500D0A0052393920484F4D45205820C7
:10A632004F4E20535441525455500D0A005239394D
:10A6420020656D657267656E63792073746F700D36
:10A652000A00523939206572726F720D0A0052383F
:10A6620032005239392073746F707065640D0A00BC
:10A67200523939206572726F7220002064656163FD
:10A68200746976617465206D6F746F7220582064EE
:10A69200756520746F206D697373656420737465CA
:10A6A2007073002064656163746976617465206DFE
:10A6B2006F746F7220592064756520746F206D6904
:10A6C20073736564207374657073002064656163DD
:10A6D200746976617465206D6F746F72205A20649C
:10A6E200756520746F206D6973736564207374657A
:10A6F2007073005239392074696D656F7574205812
:10A7020020617869730D0A005239392074696D65C8
:10A712006F7574205920617869730D0A00523939B6
:10A722002074696D656F7574205A20617869730DA4
:10A732000A0020510052383100205841002058426E
:10A74200002059410020594200205A4100205A421B
:10A752000020737461200020637572200020656EF2
:10A762006420002068616C662000206C656E200009
:10A77200206D696E2000206D617820002073706466
:10A7820020005239392057696C6C207A65726F202B
:10A7920058005239392057696C6C207A65726F20E3
:10A7A20059005239392057696C6C207A65726F20D2
:10A7B2005A00523231005000560052393920457247
:10A7C200726F723A20696E76616C69642070617290
:10A7D200616D657465722069640D0A00523431003E
:10A7E200686F6D650D0A0052323000523833200016
:10A7F2005239392043616C6962726174696F6E20EB
:10A802006572726F723A20696E76616C696420615A
:10A812007869732073656C65637465640D0A002042
:10A8220061786973200020617420737461727469A5
:10A832006E6720706F696E7400523233002063615C
:10A842006C6962726174696E67206C656E677468A8
:10A8520000207374657020636F756E743A20005225
:10A862003939206D6F76656D656E7420646F6E6523
:10A872000D0A0020617420656E6420706F696E7429
:10A88200005239392043616C6962726174696F6E7A
:10A89200206572726F723A20656E642073746F70F5
:10A8A20020616374697665206265666F72652073E4
:10A8B200746172740D0A00206D6F766520746F20CA
:10A8C200737461727420666F722063616C69627264
:10A8D2006174696F6E006E616E00696E66006F76FC
:02A8E20066000E
:00000001FF
